:100000000020001071010000350200003D020000D8
:1000100000000000000000000000000000000000E0
:100020000000000000000000000000004502000089
:1000300000000000000000004D020000550200001A
:100040005D0200005D0200005D0200005D02000034
:100050005D0200005D0200005D0200005D02000024
:100060005D0200005D0200000000000000000000D2
:1000700000000000000000005D0200005D020000C2
:100080005D0200005D0200005D0200005D020000F4
:100090005D0200005D0200000000000000000000A2
:1000A0005D0200005D0200005D0200005D020000D4
:1000B0000000000000000000000000000000000040
:1000C0007864000000000010440000007864000024
:1000D00000000020000000007864000000400020C4
:1000E000000000004400001000020000000000209A
:1000F00000000000004000200000000080B588B033
:1001000000AFF860B9607A60BB68FB61FB68BB61F7
:1001100000237B610AE0FB691A1DFA61BA69111DAF
:10012000B96112681A607B6904337B617A697B6804
:100130009A42F0D3BD4608B080BDC04680B584B0B9
:1001400000AF786039607B68FB600023BB6007E02C
:10015000FB681A1DFA6000221A60BB680433BB609A
:10016000BA683B689A42F3D3BD4604B080BDC0462E
:1001700080B586B000AF284B3B613B691B68C0224D
:1001800012051A433B691A60244B7B6116E07B69B8
:100190001A1D7A611B68FB607B691A1D7A611B68F6
:1001A000BB607B691A1D7A611B687B60F968BA685D
:1001B0007B68081C111C1A1CFFF7A0FF7A69184BFA
:1001C0009A42E4D30FE07B691A1D7A611B68BB6019
:1001D0007B691A1D7A611B687B60BA687B68101C9A
:1001E000191CFFF7ABFF7A690E4B9A42EBD30E4B0B
:1001F0001B6810331B683B603B681B681A1C0B4B69
:100200001A603B6804331B681A1C094B1A6002F021
:10021000CBF803F08DFAFEE780800440C0000000B8
:10022000E4000000FC000000F81FFF1FF0000010B9
:10023000EC00001080B500AFFEE7C04680B500AF0F
:10024000FEE7C04680B500AFFEE7C04680B500AF10
:10025000FEE7C04680B500AFFEE7C04680B500AF00
:10026000FEE7C046FFFFFFFFFFFFFFFFFFFFFFFFAF
:10027000FFFFFFFFFFFFFFFFFFFFFFFFFFFFFFFF8E
:10028000FFFFFFFFFFFFFFFFFFFFFFFFFFFFFFFF7E
:10029000FFFFFFFFFFFFFFFFFFFFFFFFFFFFFFFF6E
:1002A000FFFFFFFFFFFFFFFFFFFFFFFFFFFFFFFF5E
:1002B000FFFFFFFFFFFFFFFFFFFFFFFFFFFFFFFF4E
:1002C000FFFFFFFFFFFFFFFFFFFFFFFFFFFFFFFF3E
:1002D000FFFFFFFFFFFFFFFFFFFFFFFFFFFFFFFF2E
:1002E000FFFFFFFFFFFFFFFFFFFFFFFFFFFFFFFF1E
:1002F000FFFFFFFFFFFFFFFFFFFFFFFFFFFFFFFF0E
:1003000090B585B000AF78602D4B9B6898472C4B1B
:100310001B6998472A4B1B6A002B03D0284B5B6A4A
:10032000002B1AD1264BDB697968FF2212040A40A0
:10033000120CD2B2101C9847214BDB697968FF225E
:1003400012020A40120AD2B2101C98471C4BDB69F9
:100350007A68D2B2101C98471DE07A68FF231B040C
:1003600013401B0CDAB23B1C0C331A707A68FF2363
:100370001B0213401B0ADAB23B1C0C335A707B6819
:10038000DAB23B1C0C339A700D4B5B6A3A1C0C3290
:10039000101C032198470A4B9B693C1C0F3498475B
:1003A000031C2370064B5B699847054BDB68984735
:1003B0003B1C0F331B78181CBD4605B090BDC046D2
:1003C0000000001080B584B000AF78600A1CFB1CF0
:1003D0001A702D4B9B6898472B4B1B6998477B687D
:1003E000042213437B60284B5B6A002B20D1264BF1
:1003F000DB697968FF2212040A40120CD2B2101C89
:100400009847214BDB697968FF2212020A40120AE1
:10041000D2B2101C98471C4BDB697A68D2B2101C10
:100420009847194BDB69FA1C1278101C984722E098
:100430007A68FF231B0413401B0CDAB23B1C0C33FD
:100440001A707A68FF231B0213401B0ADAB23B1CA6
:100450000C335A707B68DAB23B1C0C339A703B1C2D
:100460000C33FA1C1278DA70074B5B6A3A1C0C32B8
:10047000101C04219847044B5B699847024BDB68CA
:100480009847BD4604B080BD0000001090B587B00D
:1004900000AFF860B960BB1D1A803A4B9B68984763
:1004A000384B1B699847374B1B6A002B03D0354BE1
:1004B0005B6A002B37D1334BDB69F968FF221204EA
:1004C0000A40120CD2B2101C98472E4BDB69F96817
:1004D000FF2212020A40120AD2B2101C9847294B7E
:1004E000DB69FA68D2B2101C98473B1C1633002215
:1004F0001A8010E03B1C16331B88BA68D418214BB5
:100500009B699847031C23703B1C16331A883B1CBD
:10051000163301321A803A1C1632BB1D12881B8812
:100520009A42E7D325E0FA68FF231B0413401B0C13
:10053000DAB23B1C10331A70FA68FF231B02134017
:100540001B0ADAB23B1C10335A70FB68DAB23B1C50
:1005500010339A700B4B5B6A3A1C1032101C03214B
:100560009847084B1B6AB968BA1D1288081C111CF1
:100570009847044B5B699847024BDB689847BD4638
:1005800007B090BD0000001080B586B000AFF860E5
:10059000B960BB1D1A803A4B9B689847384B1B6962
:1005A0009847FB6804221343FB60354B5B6A002BC2
:1005B00037D1334BDB69F968FF2212040A40120C71
:1005C000D2B2101C98472E4BDB69F968FF22120249
:1005D0000A40120AD2B2101C9847294BDB69FA680C
:1005E000D2B2101C98473B1C163300221A8010E030
:1005F000234BDB693A1C16321288B9688A181278C4
:10060000101C98473B1C16331A883B1C16330132CA
:100610001A803A1C1632BB1D12881B889A42E7D3F7
:1006200025E0FA68FF231B0413401B0CDAB23B1CC5
:1006300010331A70FA68FF231B0213401B0ADAB248
:100640003B1C10335A70FB68DAB23B1C10339A70B3
:100650000B4B5B6A3A1C1032101C03219847084B65
:100660005B6AB968BA1D1288081C111C9847044BB4
:100670005B699847024BDB689847BD4606B080BD72
:100680000000001090B585B000AF021CFB1D1A7071
:100690003B1C0E3300221A803B1C0C3300221A80B4
:1006A000FB1D1B789B000133DB00802292019B180D
:1006B000181CFFF725FE031C1A1C3B1C0C331A8068
:1006C0003B1C0C331B881B029CB2FB1D1B789B0040
:1006D0000133DB00842292019B18181CFFF710FEE7
:1006E000031C1A1C3B1C0C33A2181A803B1C0C3335
:1006F0001B88002B25D0FB1D1B789B000133DB00E2
:10070000802292019B18181CFFF7FAFD031C1A1C8B
:100710003B1C0E331A803B1C0E331B881B029CB201
:10072000FB1D1B789B000133DB00842292019B1888
:10073000181CFFF7E5FD031C1A1C3B1C0E33A21806
:100740001A803A1C0E323B1C0C3312881B889A42CA
:10075000A6D13B1C0E331B88181CBD4605B090BDAE
:1007600090B585B000AF021CFB1D1A703B1C0E3308
:1007700000221A803B1C0C3300221A80FB1D1B78C0
:100780009B000133DB00982292019B18181CFFF795
:10079000B7FD031C1A1C3B1C0C331A803B1C0C338A
:1007A0001B881B029CB2FB1D1B789B000133DB00E6
:1007B0009C2292019B18181CFFF7A2FD031C1A1C17
:1007C0003B1C0C33A2181A803B1C0C331B88002BDB
:1007D00025D0FB1D1B789B000133DB009822920182
:1007E0009B18181CFFF78CFD031C1A1C3B1C0E33B6
:1007F0001A803B1C0E331B881B029CB2FB1D1B780E
:100800009B000133DB009C2292019B18181CFFF710
:1008100077FD031C1A1C3B1C0E33A2181A803A1CCD
:100820000E323B1C0C3312881B889A42A6D13B1C0B
:100830000E331B88181CBD4605B090BD90B585B021
:1008400000AF3960FB1D011C19703B1D1A803B1C59
:100850000E3300221A800023BB603B1D1B88002B37
:1008600000D15FE0FB1D1B789B000133DB00902271
:1008700092019B18181CFFF743FD031C1B029CB23E
:10088000FB1D1B789B000133DB00942292019B1817
:10089000181CFFF735FD031C1A1C3B1C0E33A21855
:1008A0001A803B1C0E331B881A02FB1D1B789B0011
:1008B0000233DB00D318BB60B9683A683B1D1B8864
:1008C000081C111C1A1CFFF75FFE3B1C0E33391C61
:1008D0000E313A1D098812888A181A80FB1D1B7870
:1008E0009B000133DB00902292019B181A1C3B1CD9
:1008F0000E331B881B0A9BB2DBB2101C191CFFF7BE
:1009000061FDFB1D1B789B000133DB0094229201EB
:100910009B181A1C3B1C0E331B88DBB2101C191CC5
:10092000FFF750FDBD4605B090BDC04690B585B0FF
:1009300000AF3960FB1D011C19703B1D1A803B1C68
:100940000E3300221A800023BB603B1D1B88002B46
:1009500000D15FE0FB1D1B789B000133DB00A02270
:1009600092019B18181CFFF7CBFC031C1B029CB2C6
:10097000FB1D1B789B000133DB00A42292019B1816
:10098000181CFFF7BDFC031C1A1C3B1C0E33A218DD
:100990001A803B1C0E331B881A02FB1D1B789B0020
:1009A0000333DB00D318BB60B9683A683B1D1B8872
:1009B000081C111C1A1CFFF769FD3B1C0E33391C67
:1009C0000E313A1D098812888A181A80FB1D1B787F
:1009D0009B000133DB00A02292019B181A1C3B1CD8
:1009E0000E331B881B0A9BB2DBB2101C191CFFF7CD
:1009F000E9FCFB1D1B789B000133DB00A422920164
:100A00009B181A1C3B1C0E331B88DBB2101C191CD4
:100A1000FFF7D8FCBD4605B090BDC04680B588B094
:100A200000AFF860B9607A607B68062B02D10123C1
:100A3000BB6107E07B68112B02D10223BB6101E09F
:100A40000123BB610023FB610EE0FB69DBB2181CD4
:100A5000FFF786FE031C002B03D1FB69072B00DC8C
:100A600005E0FB690133FB61FB69082BEDDDFB69E8
:100A7000072B02DD01235B421BE0FB69D9B2BB6996
:100A8000DAB2FB699BB20D481B189BB2081C111C03
:100A90001A1C002300F0AAFE031C7B61FB69074AB5
:100AA0009B180749FA69081C111C1A1C03F0B2FBB9
:100AB0007B69181CBD4608B080BDC0468813000085
:100AC0005061000080B584B000AF78607B68DBB215
:100AD000181C00F0B9FF031CFB60FB68181CBD4626
:100AE00004B080BD80B584B000AF786039607B68A9
:100AF000DBB2181C01F024F8031CFB60FB68181C17
:100B0000BD4604B080BDC04680B586B000AFF86079
:100B1000B9607A603B60FB68D9B27B689BB2BA6807
:100B2000081C111C1A1C01F0B7F9031C7B617B69BE
:100B3000181CBD4606B080BD80B586B000AFF86019
:100B4000B9607A603B60FB68D9B27B689BB2BA68D7
:100B5000081C111C1A1C01F061F8031C7B617B69E5
:100B6000181CBD4606B080BD80B500AFBD4680BD37
:100B700080B500AFBD4680BD80B500AFBD4680BD2D
:100B800080B500AFBD4680BD80B582B000AF786053
:100B90007B681B78DBB2181CBD4602B080BDC04626
:100BA00080B582B000AF78600A1CFB1C1A707B68AD
:100BB000FA1C12781A70BD4602B080BD80B500AF35
:100BC0000023181CBD4680BD80B582B000AF021C5A
:100BD000FB1D1A70BD4602B080BDC04680B582B014
:100BE00000AF78600A1CBB1C1A80BD4602B080BDF5
:100BF00080B582B000AF78600A1CBB1C1A80BD466D
:100C000002B080BD80B582B000AF786039607B688B
:100C1000002B02D03B68002B06D1084B084A1A6112
:100C2000064B084A5A6105E0044B7A681A61034B87
:100C30003A685A61BD4602B080BDC046000000104F
:100C4000790B0000810B000080B582B000AF7860A6
:100C50003960C0460E4B1B881A1C80239B00134032
:100C6000F8D07B68002B02D03B68002B06D1084BE4
:100C7000084A9A61064B084ADA6105E0044B7A6833
:100C80009A61034B3A68DA61BD4602B080BDC04646
:100C900000000010BD0B0000C90B000080B582B041
:100CA00000AF78603960C0460E4B1B881A1C802349
:100CB0009B001340F8D07B68002B02D03B68002BD0
:100CC00006D1084B084A1A62064B084A5A6205E0E8
:100CD000044B7A681A62034B3A685A62BD4602B006
:100CE00080BDC04600000010DD0B0000F10B0000CD
:100CF00090B587B000AF021C3960FB1D1A703B1C19
:100D0000173300221A703B1C0C3300221A603B1C64
:100D10000C3300225A60FB1D1B780F2B00D9BDE05D
:100D20009A00634BD3181B689F4600F001F9B8E0A6
:100D30003B68002B0BD03B1C0C333A681A603B1C01
:100D40000C331B681A1C08323B1C0C335A603B1CCA
:100D50000C331A683B1C0C335B68101C191C00F028
:100D60003BF9031C9EE03B681B88181C00F0F6F959
:100D700097E000F01DFA031C1A1C3B681A8090E0F3
:100D80003B681B88181C00F047FA8AE000F06CFAF8
:100D9000031C1A1C3B681A8083E03B681B881B0AF3
:100DA0009BB2DBB298225201101C191CFFF70AFB00
:100DB0003B681B88DBB2A0225201101C191CFFF7F4
:100DC00001FB6EE098235B01181CFFF799FA031CE6
:100DD0001B029CB2A0235B01181CFFF791FA031CB5
:100DE000E3189AB23B681A805BE0324B9A783B6812
:100DF0001A703B6801332F4AD2781A703B6802336D
:100E00002C4A12791A703B6803332A4A52791A70B5
:100E10003B680433274A92791A703B6805330022F5
:100E20001A703EE000F08AFA3BE03B68181C00F0C4
:100E3000B9FA36E03B68181C00F01AFB31E03B6859
:100E40001B78181C00F06AFB031C2BE000F058FA1A
:100E5000031C1A1C3B1C17331A703B1C17331B78DE
:100E6000FF2B01D1FF231DE03B683A1C173212789B
:100E70001A7016E000F028FA031C1A1C3B1C1733EA
:100E80001A703B1C17331B78FF2B01D1FF2309E09D
:100E90003B683A1C173212781A7002E0FF2301E017
:100EA000C04600235BB2181CBD4607B090BDC046CB
:100EB000686100000000001080B582B000AF021C25
:100EC0003960FB1D1A70FB1D1B78052B26D89A0074
:100ED000164BD3181B689F463B68181C00F084FB18
:100EE0001EE03B68181C00F0C1FB19E03B681B7852
:100EF000181C00F0FDFB031C13E000F027FC031C92
:100F00001A1C3B681A700BE03B68181C00F028FCA8
:100F100006E03B68181C00F047FC01E0FF2300E0FE
:100F200000235BB2181CBD4602B080BDA861000062
:100F300080B586B000AF90231A013B1D101C191C10
:100F40000622FFF7A3FA80235A003B1C1433101C1F
:100F5000191C0422FFF79AFAA023DA003B1C103375
:100F6000101C191C0422FFF791FAF0231A013B1CF4
:100F70000C33101C191C0422FFF788FA0020802172
:100F8000FFF720FA0020FFF7BBF990231A013B1D61
:100F9000101C191C0622FFF7F7FA80235A003B1C8D
:100FA0001433101C191C0422FFF7EEFAA023DA00F8
:100FB0003B1C1033101C191C0422FFF7E5FAF02328
:100FC0001A013B1C0C33101C191C0422FFF7DCFA1D
:100FD000BD4606B080BDC04680B584B000AF786025
:100FE00039603B1C0E3300221A70FFF7A1FF7B68AB
:100FF000002B54D03B1C0E3300221A703B1C0F33C5
:1010000000221A701DE03B1C0F331B785BB27A681C
:10101000D3181A783B1C0E331B78D318DAB23B1C5A
:101020000E331A703B1C0E331B785BB2102B01DDA4
:10103000FF238DE03B1C0F331A783B1C0F3301322A
:101040001A703B1C0F331B785BB2072BDBDD3B1C9C
:101050000F3300221A701CE03B1C0F331B785BB26D
:101060009B000133DB00F82252019B181A1C3B1C29
:101070000F331B785BB27968CB181B78101C191CD6
:10108000FFF7A0F93B1C0F331A783B1C0F330132DA
:101090001A703B1C0F331B785BB2072BDCDD3B68FF
:1010A000002B54D03B1C0E3300221A703B1C0F3314
:1010B00000221A701DE03B1C0F331B785BB23A68AC
:1010C000D3181A783B1C0E331B78D318DAB23B1CAA
:1010D0000E331A703B1C0E331B785BB2102B01DDF4
:1010E000FF2335E03B1C0F331A783B1C0F330132D2
:1010F0001A703B1C0F331B785BB2072BDBDD3B1CEC
:101100000F3300221A701CE03B1C0F331B785BB2BC
:101110009B000133DB00F02252019B181A1C3B1C80
:101120000F331B785BB23968CB181B78101C191C65
:10113000FFF748F93B1C0F331A783B1C0F33013281
:101140001A703B1C0F331B785BB2072BDCDD0023CE
:101150005BB2181CBD4604B080BDC04680B584B0EB
:1011600000AF021CBB1D1A803B1C0F33BA1D128836
:101170001A70BB1D1B881B0A9AB23B1C0E331A70D7
:101180003B1C0F331B780F229343DBB2A822520182
:10119000101C191CFFF716F9B8235A013B1C0E331B
:1011A0001B78101C191CFFF70DF9BD4604B080BD5B
:1011B00090B583B000AFFB1D00221A70BB1D00224A
:1011C0001A703B1D00221A80A8235B01181CFFF730
:1011D00097F8031C1A1CFB1D0F218A431A70BC1DB3
:1011E000B8235B01181CFFF78BF8031C23703B1D11
:1011F000BA1D12781A803B1D1B881B0299B2FB1D79
:101200001B789AB23B1D8A181A803B1D1B88181C3C
:10121000BD4603B090BDC04680B584B000AF021C8F
:10122000BB1D1A803B1C0F33BA1D12881A70BB1DE0
:101230001B881B0A9AB23B1C0E331A70B0235A014A
:101240003B1C0F331B78101C191CFFF7BBF8C02385
:101250005A013B1C0E331B78101C191CFFF7B2F807
:10126000BD4604B080BDC04690B583B000AFFB1D45
:1012700000221A70BB1D00221A703B1D00221A802A
:10128000FC1DB0235B01181CFFF73AF8031C237008
:10129000BC1DC0235B01181CFFF732F8031C237030
:1012A0003B1DBA1D12781A803B1D1B881B0299B288
:1012B000FB1D1B789AB23B1D8A181A803B1D1B88A8
:1012C000181CBD4603B090BD80B582B000AFB823F6
:1012D0009B01181CFFF714F8031C1A1C0123134070
:1012E00003D0FB1D01221A7002E0FB1D00221A70C0
:1012F000FB1D1B785BB2181CBD4602B080BDC0460A
:1013000080B582B000AFFB1D00221A70B8239B018C
:10131000181CFEF7F5FF031C1A1C3023134003D0E2
:10132000FB1D01221A7002E0FB1D00221A70FB1D3A
:101330001B785BB2181CBD4602B080BD90B583B06F
:1013400000AFFC1DB8239B01181CFEF7D9FF031C3E
:101350002370FB1DFA1D11787F220A401A70B823F2
:101360009A01FB1D1B78101C191CFFF72BF8FC1DA4
:10137000B8239B01181CFEF7C3FF031C2370FB1D41
:10138000FA1D1278802149420A431A70B8239A0143
:10139000FB1D1B78101C191CFFF714F8BD4603B089
:1013A00090BDC04680B584B000AF78603B1C0F3361
:1013B00000221A707B681B78012B08D13B1C0F336D
:1013C0003A1C0F32127840210A431A7007E03B1C86
:1013D0000F333A1C0F32127840218A431A707B680F
:1013E0005B78012B08D13B1C0F333A1C0F3212786B
:1013F00038210A431A702CE07B68DB78012B15D169
:101400007B689B78012B08D13B1C0F333A1C0F32B1
:10141000127818210A431A701BE03B1C0F333A1C48
:101420000F32127808210A431A7012E07B689B7809
:10143000012B08D13B1C0F333A1C0F3212781021BC
:101440000A431A7005E03B1C0F333A1C0F32127826
:101450001A70B8239A013B1C0F331B78101C191CFF
:10146000FEF7B0FFFFF76AFFBD4604B080BDC0467F
:1014700090B585B000AF78603B1C0F3300221A7026
:101480003C1C0F34B8239B01181CFEF739FF031CCA
:1014900023703B1C0F331A78402313405A1E93418C
:1014A000DBB21A1C7B681A703B1C0F331A78382386
:1014B0001340202B01D0382B03D17B6801225A70B6
:1014C00003E07B6800225A70C0463B1C0F331A7839
:1014D00038231340182B03D0202B01D0102B03D11D
:1014E0007B6801229A7003E07B6800229A70C046F4
:1014F0003B1C0F331A7838231340182B03D0202BB2
:1015000001D0082B03D17B680122DA7003E07B68ED
:101510000022DA70C046BD4605B090BD90B585B0DA
:1015200000AF021CFB1D1A703B1C0F3300221A7007
:101530003C1C0F34B8239B01181CFEF7E1FE031C72
:1015400023703B1C0F331A784023134001D1FF2333
:1015500045E03B1C0F333A1C0F32127838218A4386
:101560001A70FB1D1B78012B08D13B1C0F333A1C52
:101570000F32127830210A431A7007E03B1C0F33F8
:101580003A1C0F32127838210A431A70B8239A0194
:101590003B1C0F331B78101C191CFEF713FFFFF7C1
:1015A000CDFE3C1C0F34B8239B01181CFEF7A8FE8F
:1015B000031C2370FB1D1B78012B07D13B1C0F3331
:1015C0001A783023134009D0002308E03B1C0F3366
:1015D0001A783823134001D0002300E0FF235BB2C8
:1015E000181CBD4605B090BD80B582B000AF7860D4
:1015F0007B6890221201101C191C0622FEF7C4FF02
:101600007B680E3380225200101C191C0422FEF746
:10161000BBFF7B680A33A022D200101C191C0422D5
:10162000FEF7B2FF7B680633F0221201101C191C72
:101630000422FEF7A9FF7B689A7C0A4B1A707B682C
:10164000DA7C084B5A707B681A7D064B9A707B686F
:101650005A7D044BDA707B689A7D034B1A70BD4645
:1016600002B080BD440000104800001080B582B078
:1016700000AF78607B6890221201101C191C0622B2
:10168000FEF704FF7B680E3380225200101C191CE9
:101690000422FEF7FBFE7B680A33A022D200101C56
:1016A000191C0422FEF7F2FE7B680633F0221201B9
:1016B000101C191C0422FEF7E9FE0B4B1A787B68FC
:1016C0009A74094B5A787B68DA74074B9A787B686E
:1016D0001A75054BDA787B685A75044B1A787B6863
:1016E0009A75BD4602B080BD44000010480000104D
:1016F00090B585B000AF021CFB1D1A703B1C0F3368
:1017000000221A70FB1D1B783A22934301D0FF235D
:1017100017E03C1C0F340020FEF7F2FD031C237081
:101720003B1C0F33391C0F31FA1D097812780A431C
:101730001A703B1C0F331B780020191CFEF742FE69
:1017400000235BB2181CBD4605B090BD80B500AF4C
:101750000020FEF7D5FD031C181CBD4680BDC04609
:1017600080B582B000AF78607B681B78D8225201C8
:10177000101C191CFEF726FE7B685B881B0A9BB2B7
:10178000DBB2C8225201101C191CFEF71BFE7B683D
:101790005B88DBB2D0225201101C191CFEF712FE2E
:1017A000BD4602B080BDC04690B583B000AF786042
:1017B000D8235B01181CFEF7A3FD031C1A1C7B68D1
:1017C0001A70C8235B01181CFEF79AFD031C1B024C
:1017D0009CB2D0235B01181CFEF792FD031CE3189A
:1017E0009AB27B685A80BD4603B090BD90B585B073
:1017F00000AF041C081C111C1A1CFB1D1C70BB1D17
:1018000018703B1D1980FB1C1A70FB1D1B78082BE0
:1018100001D9FF2304E1BB1D1B78022B14D0042B3C
:1018200012D0012B0ED1F0231A013B1C0C33101CDB
:10183000191C0422FEF72AFEFB68002B01D1FD23B0
:10184000EEE001E0FB23EBE0C046FB1C1A7804232A
:10185000134001D0FA23E3E0FB1C1B78002B27D0B8
:10186000BB1D1B78012B02D0022B08D020E0FB1CF3
:101870001A782123134001D1FA23D1E018E0FB1C90
:101880001A782023134006D0FB1C1B785BB2002B78
:1018900001DBFA23C4E0FB1C1A781023134006D0A6
:1018A000FB1C1B785BB2002B01DBFA23B8E0C046BF
:1018B000FB1D1B78181C00F0C7F8FB1D1B789B0054
:1018C0000133DB001A1CFB1C1B780F218B43D9B2A0
:1018D000BB1D1B780B43DBB2DBB2101C191CFEF7DF
:1018E00071FD3B1D1B88002B0FD1504B1B885A1CD0
:1018F00091B24E4A11803A1D13804C4B1A884C4BC2
:101900009A4202D1494B4B4A1A80FB1D1B789B001F
:101910000133DB008021C9005B181A1C3B1D1B88AA
:101920001B0A9BB2DBB2101C191CFEF74BFDFB1D02
:101930001B789B000133DB00A022D2009B181A1CED
:101940003B1D1B88DBB2101C191CFEF73BFDFB1D69
:101950001B789B000133DB000133FF33181C01218E
:10196000FEF730FDC046FB1D1B789B000133DB00FA
:101970000133FF33181CFEF7C3FC031C002BF2D10C
:10198000FB1D1B780122111C99400B1C9BB2DB43F1
:101990009BB2294A128892B213409BB29AB2264B4C
:1019A0001A80FB1C1A7801231A40FB1D1B78111C9E
:1019B00099400B1C9AB2204B1B889BB213439BB2DD
:1019C0009AB21D4B1A80FB1D1B780122111C9940F5
:1019D0000B1C9BB2DB439BB2184A128892B2134095
:1019E0009BB29AB2154B1A80FB1D1A78144B520009
:1019F0000021D152FB1D1B78124A0021D154C04650
:101A0000FB1D1B789B000133DB00C02292009B185A
:101A1000181CFEF775FC031C002BF1D0FB1D1B7876
:101A20005BB2181CBD4605B090BDC0462800001032
:101A3000F0FF000000C0FFFF4A0000104C00001043
:101A4000500000106000001080B582B000AF021C92
:101A5000FB1D1A70FB1D1B78082B01D9FF2361E0C9
:101A6000FB1D1B789B000133DB000133FF33181C87
:101A70001021FEF7A7FCC046FB1D1B789B0001331D
:101A8000DB000133FF33181CFEF73AFC031C002B6C
:101A9000F2D1FB1D1B789B000133DB008021890004
:101AA0005B18181C1F21FEF78DFCFB1D1B78012203
:101AB000111C99400B1C9BB2DB439BB21C4A128841
:101AC00092B213409BB29AB2194B1A80FB1D1B783D
:101AD0000122111C99400B1C9BB2DB439BB2154A9F
:101AE000128892B213409BB29AB2124B1A80FB1D1D
:101AF0001A78114B52000021D152FB1D1B780F4A5E
:101B00000021D154C046FB1D1B789B000133DB0034
:101B1000C02292009B18181CFEF7F2FB031C002B3E
:101B2000F1D101235BB2181CBD4602B080BDC04696
:101B30004A0000104C00001050000010600000101F
:101B400080B582B000AF021CFB1D1A70FB1D1B7814
:101B5000082B01D9FF235CE0FB1D1B789B000133A0
:101B6000DB00181CFEF7CCFB031C1A1C0F231340D0
:101B7000012B01D0FB234CE0FB1D1B789B000133A4
:101B8000DB00C02292009B18181CFEF7B9FB031C57
:101B9000132B01D0FD233CE0FB1D1B789B00013380
:101BA000DB000133FF33181C0221FEF70BFCC0469B
:101BB000FB1D1B789B000133DB000133FF33181C36
:101BC000FEF79EFB031C002BF2D113E0FB1D1B78DC
:101BD0009B000133DB000133FF33181CFEF790FB41
:101BE000031C002B06D1FB1D1B78181CFFF72CFFD4
:101BF000FC230EE0FB1D1B789B000133DB00C022A1
:101C000092009B18181CFEF77BFB031C142BDDD1E4
:101C100001235BB2181CBD4602B080BD90B585B0F3
:101C200000AF3960FB1D011C19703B1D1A803B1C65
:101C30000F3300221A703B1C0C3300221A80FB1D4C
:101C40001B78082B02D901235B421CE1FB1D1B788A
:101C50009B000133DB00181CFEF752FB031C1A1C0F
:101C60000F231340012B02D005235B420BE13B1DE8
:101C70001B88002B02D10E235B4204E1FB1D1B7865
:101C80009B000133DB00C02189005B183C1C0F3432
:101C9000181CFEF735FB031C23703B1C0F331B780D
:101CA000172B07D03B1C0F331B781C2B02D00723AC
:101CB0005B42E8E0764B1B881A1CFB1D1B781A411F
:101CC0000123134045D0FB1D1B789B000133DB0033
:101CD000802292009B18181CFEF712FB031C191C93
:101CE0003B1C0F331F220A401A703B1C0F331A781B
:101CF000102313401DD0FB1D1B789B000133DB001C
:101D0000802189005B18181C1021FEF75BFBFB1D6E
:101D10001B780122111C99400B1C9BB2DB439BB228
:101D20005B4A128892B213409BB29AB2584B1A8007
:101D30000FE03B1C0F331A780823134007D0FB1D1C
:101D40001B78181CFFF780FE0D235B429BE00023ED
:101D500099E0FB1D1B789B000133DB00F822520148
:101D60009B18181CFEF7CCFA031C1A1C3B1C0C33E6
:101D700092021A803A1D3B1C0C3312881B889A422F
:101D800004D93B1D3A1C0C3212881A803C1C0C34BE
:101D9000FB1D1B78181CFEF775FC031C2380FB1D24
:101DA0001B789B000133DB00C02189005B183C1CC1
:101DB0000F34181CFEF7A4FA031C23703B1C0F33CE
:101DC0001B78172B0CD03B1C0F331B781C2B07D018
:101DD000FB1D1B78181CFFF737FE07235B4252E000
:101DE0002C4B1B881A1CFB1D1B781A410123134026
:101DF00008D03A1D3B1C0C3312881B889A4201D92B
:101E0000002340E03A1D3B1C0C3312881B889A4289
:101E100016D8C046FB1D19783A683B1D1B88081C64
:101E2000111C1A1CFEF70AFDFB1D1B789B000133D9
:101E3000DB000133FF33181C2021FEF7C3FA04E056
:101E40003B1D3A1D12881A80A0E7FB1D1B789B00E2
:101E50000133DB000133FF33181CFEF751FA031C7A
:101E6000002BF2D1FB1D1B780122111C99400B1C89
:101E70009AB2074B1B889BB213439BB29AB2044B96
:101E80001A803B1D1B88181CBD4605B090BDC0467E
:101E90004C0000104A00001090B585B000AF3960CA
:101EA000FB1D011C19703B1D1A803B1C0F330022C7
:101EB0001A703B1C0C3300221A80FB1D1B78082B68
:101EC00002D901235B42CEE0FB1D1B789B0001334E
:101ED000DB00181CFEF714FA031C1A1C0F23134016
:101EE000012B02D005235B42BDE03B1D1B88002B6C
:101EF00002D10E235B42B6E0FB1D1B789B00013331
:101F0000DB00F02252019B18181CFEF7F9F9031CA4
:101F10001A1C3B1C0C3392021A803A1C0C323B1DDB
:101F200012881B889A4204D23B1D3A1C0C3212883C
:101F30001A803C1C0C34FB1D1B78181CFEF710FC8F
:101F4000031C2380FB1D1B789B000133DB00C02298
:101F500092009B183C1C0F34181CFEF7D1F9031C8F
:101F600023703B1C0F331B78172B30D03B1C0F33D7
:101F70001B781C2B23D13B1C0C331B88002B00D05F
:101F800040E0FB1D1B78181CFEF77CFB031C1C1C8F
:101F9000FB1D1B789B000133DB00F82252019B18CC
:101FA000181CFEF7ADF9031C9B029C420FD1FB1DD0
:101FB0001B78181CFFF748FD07235B4253E0FB1D0D
:101FC0001B78181CFFF740FD07235B424BE0284BB2
:101FD0001B881A1CFB1D1B781A410123134006D0D5
:101FE0003B1C0C331B88002B01D100233BE03B1C26
:101FF0000C331B88002B00D004E03B1D3A1D1288D7
:102000001A8096E73A1C0C323B1D12881B889A42B4
:1020100004D23B1D3A1C0C3212881A80FB1D197821
:102020003A683B1D1B88081C111C1A1CFEF77EFC1D
:10203000FB1D1B789B000133DB000133FF33181CB1
:102040004021FEF7BFF9C046FB1D1B789B00013302
:10205000DB000133FF33181CFEF752F9031C002B81
:10206000F2D13B1D1B88181CBD4605B090BDC04673
:102070004A00001090B587B000AF78603B1C143365
:1020800000221A803B1C163300221A8002200121F4
:102090000622FEF7C3FC031C3B613B69013307D1F9
:1020A0003C4A3B69101C191C02F0B4F83B696CE017
:1020B0003B1C0F333A691A703B1C0F331B78181CFA
:1020C0000421FEF70FFD031C3B613B69012B01D08E
:1020D0003B695AE03C1C14343B1C0F331B78181C22
:1020E000FEF73EFB031C23803B1C14331B88002B94
:1020F0004AD03B1C0F3319783B1C14331B887A6879
:10210000081C111C1A1C0023FEF7FEFC031C3B617B
:102110003B69002B00DC37E03B1C163300221A80A1
:102120002AE03B1C0F3319783B1C16331B887A6856
:10213000D2183B1C143318883B1C16331B88C31A57
:10214000081C111C1A1C0023FEF7F6FC031C3B6143
:102150003B69002B07DA3B1C0F331B78181CFEF77A
:10216000B1FC3B6911E03B6999B23B1C16333A1C48
:10217000163212888A181A803A1C14323B1C163305
:1021800012881B889A42CCD1A4E7181CBD4607B020
:1021900090BDC046C061000080B582B000AF7860DD
:1021A0007B685B6802221A437B685A60BD4602B0B6
:1021B00080BDC04680B584B000AFF860B9607A6079
:1021C0003B60FB681B68FF22191C91430A1CBB681B
:1021D0001A437B681A433B681A43FB681A60BD4682
:1021E00004B080BD90B583B000AF7860FB1C19705F
:1021F000BB1C1A70FB1C1A78FB1C19787B688020AA
:10220000000109188900C958BB1C1B780120041C57
:102210009C40231C19437B68802000011218920007
:10222000D150BD4603B090BD80B500AF154B181C12
:1022300000210622822300F06BFD124B181C0021A6
:102240000822812300F064FD0E4B181C0021092296
:10225000812300F05DFD0B4B181C0021022210238E
:1022600000F056FDA023DB05181C00210222FFF719
:10227000B9FFA023DB05181C00210322FFF7B2FFE2
:10228000BD4680BD0040044080B500AFFFF7CCFFE5
:102290000D4B181C01F0B4F80B4B181C0721002241
:1022A000C023FFF787FF084B181C012101F052F8EB
:1022B000054A064B101C191C01F066F8024B181C4D
:1022C000FFF76AFFBD4680BD00000440002D3101CC
:1022D00080B584B002AF00F0F5FB00F011FB0020E8
:1022E000012100F0E1FA0120012100F0DDFA0220D5
:1022F000012100F0D9FAFFF7C7FF00F08BF91C4B62
:102300006A46191C103108681060888890808979A5
:102310009171186859689A68DB6800F067F93B1C8E
:1023200000221A6000229A803B1C0820191CFEF72C
:10233000DFFC104B181C01F06DFF0F4A3B1C101CFA
:10234000191C0122012301F065FF0C4B181C01F040
:1023500061FF0B4B181C01F05DFF084B181C01F0CE
:1023600059FF00F0B7F8074B181CFFF783FEFAE798
:102370002C000010D86100000462000024620000FC
:10238000506200006C00001010B5024B1B689847AB
:1023900010BDC046F000001010B5024B1B689847F6
:1023A00010BD0000EC00001080B500AF00F07EFB17
:1023B000BD4680BD80B582B000AF7860081C111C9E
:1023C0001A1CFB1C1870BB1C19707B1C1A70FB1CA0
:1023D0001878BB1C1A787B1C19787B68400182181E
:1023E000D154BD4602B080BD80B500AFA023DB054F
:1023F000181C002102220023FFF7DCFFBD4680BD30
:1024000080B500AFA023DB05181C002102220123A8
:10241000FFF7D0FFBD4680BD80B582B000AF064A51
:10242000FB1D101C191C012200F0E0FEFB1D1B7897
:10243000181CBD4602B080BD0000044080B582B0CB
:1024400000AF021CFB1D1A70044AFB1D101C191C56
:10245000012200F021FEBD4602B080BD0000044014
:1024600080B582B000AF78600A1CBB1C1A80BB1C10
:102470001B8805497A68081C111C1A1C00F0B6FE5E
:10248000BD4602B080BDC0460000044080B582B0A9
:1024900000AF78600A1CBB1C1A80BB1C1B88054956
:1024A0007A68081C111C1A1C00F0F6FDBD4602B02B
:1024B00080BDC0460000044080B582B000AF7860A7
:1024C00002E07B68013B7B607B68002BF9D1BD4655
:1024D00002B080BDF0B58DB004AF3B1C18330022B4
:1024E0001A6000229A803B1C0120191CFEF7E4FCB4
:1024F0003B1C18330820191CFEF7FAFB3B1C9B7D84
:10250000022B07D1324A3B1C1833101C191C01F056
:1025100081FE06E02F4A3B1C1833101C191C01F0E9
:1025200079FE3B1C1B78191C3B1C5B781A1C3B1C5E
:102530009B78381CC078061C381C0079051C381C98
:102540004079041C244800960195029401F062FE33
:102550003B1C9B79191C3B1CDB791A1C3B1C1B7A0E
:10256000381C407A041C1D48009401F053FE3B1CAB
:102570009B7B191C3B1CDB7B1A1C3B1C1B7C381CEB
:10258000407C041C1648009401F044FE3B1C9B7ADE
:10259000191C3B1CDB7A1A1C3B1C1B7B381C407B28
:1025A000041C1048009401F035FE3B1C9B7C191C58
:1025B0003B1CDB7C1A1C3B1C1B7D381C407D041C17
:1025C0000948009401F026FEBD4609B0F0BDC046A2
:1025D0007462000098620000C0620000E8620000BF
:1025E000FC620000106300002463000084B098B512
:1025F00000AF3C1C103420606160A260E3603B1CB3
:1026000010330020191CFEF757FCBD4698BC08BCCF
:1026100004B0184780B584B000AF3A1C214B111CA0
:102620001A1C1023081C111C1A1C01F08AF8A02384
:10263000DB05181C002103220023FFF7BBFE1A4B09
:10264000181CFFF739FFA023DB05181C002103220B
:102650000123FFF7AFFE154B181CFFF72DFF144A9F
:10266000144B101C191CFEF7CDFA134A134B101C07
:10267000191CFEF7E9FA124A124B101C191CFEF73E
:102680000DFB3B1C0120191CFEF732FB031C013320
:1026900004D10D4B181C01F0BDFDFEE7BD4604B092
:1026A00080BDC0465463000088130000102700005E
:1026B000E923000001240000192400003D2400004B
:1026C000612400008D2400003863000080B582B0D2
:1026D00000AF78607B6880221A63BD4602B080BD7F
:1026E00080B582B000AF786039607B683A689A60E4
:1026F000BD4602B080BDC04680B582B000AF7860F4
:1027000039607B683A68DA60BD4602B080BDC04679
:1027100080B582B000AF7860081C111C1A1CFB1C2D
:102720001870BB1C19707B1C1A70FB1C1878BB1C22
:102730001A787B1C19787B6840018218D154BD46F9
:1027400002B080BD90B583B000AF7860FB1C1970FB
:10275000BB1C1A70FB1C1A78FB1C19787B68802044
:10276000000109188900C958BB1C1B780120041CF2
:102770009C40231C19437B688020000112189200A2
:10278000D150BD4603B090BD80B586B000AFF860B3
:10279000B9607A6000237B6109E0BA687B69D3186D
:1027A0001B78181C00F00CF87B6901337B617A6898
:1027B0007B699A42F1D87B68181CBD4606B080BD83
:1027C00080B582B000AF021CFB1D1A70044AFB1DCD
:1027D000101C191C012200F04DFFBD4602B080BD47
:1027E0000080004080B500AF144B181C002112225D
:1027F000012300F08DFA114B181C00211322012334
:1028000000F086FA0E4B181C00F0F0FE0C4AE12393
:102810005B02101C191C00F057FF094B181C032108
:10282000FFF76AFF064B181C8121FFF759FF044B85
:10283000181CFFF74BFFBD4680BDC046004004405A
:102840000080004080B582B000AF00237B6021E0B3
:10285000134A7B68D3181A7812497B68CB181B7807
:10286000A021C905081C111C1A1CFFF76BFF0C4A9C
:102870007B68D3181A780B497B68CB181B78A0218A
:10288000C905081C111C1A1C0023FFF741FF7B68B7
:1028900001337B607B68022BDADDBD4602B080BD70
:1028A000686300006C63000080B582B000AF0A1C52
:1028B000FB1D011C1970BB1D1A70FB1D1B78022B20
:1028C00017D8FB1D1B780C4AD15CFB1D1B780B4AEB
:1028D000D25CBB1D1B78581E8341DBB201204340F4
:1028E000DBB2181C01230340DBB2A020C005FFF7B8
:1028F0000FFFBD4602B080BD686300006C6300003E
:1029000080B500AFFFF76EFFA023DB05181C00F0B9
:10291000F5F9FFF797FF00200021FFF7C5FF012021
:102920000021FFF7C1FF02200021FFF7BDFFBD46D8
:1029300080BDC04680B584B000AF021CFB1D1A707C
:10294000064B1B6903229343FB60044BFA1D11786D
:10295000FA680A431A61BD4604B080BD00C0034056
:1029600080B582B000AF0A1CFB1D011C1970BB1D95
:102970001A70074BFA1D11781F221140BA1D1078EA
:102980000322024052010A439A60BD4602B080BD54
:102990000080044080B500AF044BDA680123134087
:1029A0005A1E9341DBB2181CBD4680BD0080044016
:1029B00080B582B000AF7860024B7A689A67BD46F6
:1029C00002B080BD0080044090B583B000AF021C0F
:1029D000FB1D1A70074A07498023C958FB1D1B7845
:1029E0000120041C9C40231C19438023D150BD4668
:1029F00003B090BD0080044080B582B000AF2020BD
:102A000000F04CFD00237B6002E07B6801337B60BB
:102A10007B68FF2BF9DD012000F0A8F8802000F092
:102A20001FFD03200121FFF79BFF802000F036FDF2
:102A3000C046FFF7AFFF031C01225340DBB2002B5F
:102A4000F7D10120FFF7B4FF0220FFF773FF032047
:102A500000F0A2F8BD4602B080BDC04680B582B08D
:102A600000AF1020FFF7B0FF00237B6013E00D4B99
:102A70007A689200D15C0B4A7B689B00D3185A7825
:102A800008487B689B00C3185B88074800F040F942
:102A90007B6801337B607B680E2BE8D9BD4602B0B2
:102AA00080BDC046706300000040044080B500AFA8
:102AB000FFF7A2FFFFF7D2FF1A20FFF785FFBD4601
:102AC00080BDC04680B500AF00F0EEF8021C024B9E
:102AD0001A60BD4680BDC046F400001080B500AF4E
:102AE000024B1B68181CBD4680BDC04664630000D5
:102AF00080B500AF014B181CBD4680BD001BB70060
:102B000080B584B000AF78607B685B09D9B23B1CAC
:102B10000F330F220A401A707A681F231340BB60DC
:102B20003B1C0F331A78074B9200D258BB68013315
:102B30005B00101C191CFFF72FFC031C181CBD4662
:102B400004B080BDAC63000080B584B000AF786095
:102B500039607A681F2313400133FB603B68FA68D1
:102B60005343181CBD4604B080BDC04680B582B03A
:102B700000AF021CFB1D1A70064BFA1D12781A6476
:102B8000044B00225A64034B01225A64BD4602B032
:102B900080BDC0460080044080B582B000AF021CFA
:102BA000FB1D1A70064BFA1D12781A67044B00229F
:102BB0005A67034B01225A67BD4602B080BDC0462A
:102BC0000080044080B500AF044B5B6A181CFFF71F
:102BD00097FF031C181CBD4680BDC0460080044002
:102BE00080B582B000AF0D4B1B6CDBB21A1C032307
:102BF000134002D0012B05D009E0FFF779FF031C39
:102C00007B6006E0FFF76AFF031C7B6001E00023A6
:102C10007B607B68181CBD4602B080BD008004400C
:102C200098B500AF064B9C68FFF7DAFF031C201C29
:102C3000191CFFF789FF031C181CBD4698BDC04630
:102C40000080044080B582B000AF00237B60154B4C
:102C50001B6FDBB21A1C03231340012B0DD002DCC7
:102C6000002B05D018E0022B0CD0032B0FD013E063
:102C7000FFF73EFF031C7B600EE0FFF7B1FF031C74
:102C80007B6009E0FFF79EFF031C7B6004E0FFF719
:102C9000C7FF031C7B60C0467B68181CBD4602B0A2
:102CA00080BDC0460080044080B500AFFFF7CAFF7A
:102CB000021C054B9B6F101C191CFFF76DFB031CBE
:102CC000181CBD4680BDC0460080044090B583B04E
:102CD00000AF021CFB1D1A70074A07498023C95820
:102CE000FB1D1B780120041C9C40231C19438023DE
:102CF000D150BD4603B090BD0080044080B582B085
:102D000000AF78600620FFF7E1FFBD4602B080BD4E
:102D100080B584B000AFF8607B603B1C0B3319704A
:102D20003B1C0A331A703B1C0B331B78002B07D15A
:102D30003B1C0A331A78FB6892007968D15007E08F
:102D40003B1C0A331A78FB68183292007968D1501C
:102D5000BD4604B080BDC04690B583B000AF021C34
:102D6000FB1D1A70074B074A5268F91D09780120AC
:102D7000041C8C40211CC9430A405A60BD4603B064
:102D800090BDC0460080044090B583B000AF021CE7
:102D9000FB1D1A70064B064A5168FA1D1278012075
:102DA000041C9440221C0A435A60BD4603B090BDE7
:102DB0000080044080B582B000AF021CFB1D1A7079
:102DC000FB1D1B78181CFFF7C7FFFB1D1B78181C89
:102DD000FFF7DAFFBD4602B080BDC04690B583B0B4
:102DE00000AF021CFB1D1A70074A07498023C9580F
:102DF000FB1D1B780120041C9C40231C19438023CD
:102E0000D150BD4603B090BD0080044080B582B073
:102E100000AF7860034A94237968D150BD4602B070
:102E200080BDC0460080044080B500AF024A9423B4
:102E3000D358181CBD4680BD0080044080B582B0C8
:102E400000AF7860034A9C237968D150BD4602B038
:102E500080BDC0460080044080B500AF024A9C237C
:102E6000D358181CBD4680BD0080044080B582B098
:102E700000AF78600A1CFB1C1A707B68DB68FA1CC8
:102E8000127813405A1E9341DBB2181CBD4602B0A3
:102E900080BDC04680B582B000AF78600A1CFB1CC4
:102EA0001A707B689B69FA1C127813405A1E934172
:102EB000DBB2181CBD4602B080BDC04680B582B0F2
:102EC00000AF78607B681B68DAB20F231340DBB277
:102ED000181CBD4602B080BD80B582B000AF7860DE
:102EE0000A1CFB1C1A70FB1C1A787B681A62BD4610
:102EF00002B080BD80B582B000AF78607B689B680F
:102F00009BB2181CBD4602B080BDC04680B582B0E1
:102F100000AF78600A1CBB1C1A80BB1C1A887B6837
:102F20009A60BD4602B080BD80B584B000AFF86045
:102F3000B9607A603B60FB681B68FF22191C9143F3
:102F40000A1CBB681A437B681A433B681A43FB6838
:102F50001A60BD4604B080BD80B582B000AF786015
:102F600039607B685B680422191C91430A1C3B682A
:102F70001A437B685A60BD4602B080BD80B584B0FC
:102F800000AF78607A68094B9A4204D13B1C0F333A
:102F90000B221A7003E03B1C0F3312221A703B1CE9
:102FA0000F331B78181CBD4604B080BD00000440E0
:102FB00080B584B000AF78607A68094B9A4204D13A
:102FC0003B1C0F3300221A7003E03B1C0F3302221C
:102FD0001A703B1C0F331B78181CBD4604B080BD13
:102FE0000000044080B582B000AF786039607A6834
:102FF000074B9A4204D13B68181CFFF707FF03E018
:103000003B68181CFFF71AFFBD4602B080BDC046E2
:103010000000044080B584B000AF7860FFF712FE76
:10302000031CFB607A680D4B9A4209D1FFF7FCFE46
:10303000031CF868191CFFF7AFF9031CFB6008E0DC
:10304000FFF70AFF031CF868191CFFF7A5F9031C1A
:10305000FB60FB68181CBD4604B080BD0000044046
:1030600080B586B000AFF860B9607A60FB681A6816
:10307000084B13407B61BB681B021B041A0C7B6965
:103080001A43FB681A60FB687A681A61BD4606B08D
:1030900080BDC046FF00FFFF80B588B000AFF8607C
:1030A000B9607A600023FB610023BB6103E0FB6829
:1030B000181CFFF71FFFFB68181C0421FFF7D6FE42
:1030C000031C002BF3D1FB68181C0321FFF704FF3E
:1030D000FB68181CFFF7F2FE031C072B3ED9BB68E8
:1030E0007B6132E0FB68181C0221FFF7BFFE031C66
:1030F000012B10D1FA697B689A420CD27B691B883C
:10310000FA68101C191CFFF701FF7B6902337B6111
:10311000FB690233FB61FB68181C0121FFF7BAFE53
:10312000031C012B01D100235BE006E0FB68181CA7
:10313000FFF7E0FEBB690233BB61FB68181C04218A
:10314000FFF794FE031C012BF0D0FA697B689A42CA
:10315000C8D3BA697B689A42C4D341E0BB683B617B
:1031600036E0FB68181C0221FFF780FE031C012BD0
:1031700010D1FA697B689A420CD23B691B78FA68D5
:10318000101C191CFFF7C2FE3B6901333B61FB6950
:103190000133FB61FB68181C0121FFF77BFE031C58
:1031A000012B01D100231CE006E0FB68181CFFF78F
:1031B000A1FEBB690133BB61FB68181C0421FFF74A
:1031C00055FE031C012B03D1BA697B689A42ECD3EC
:1031D000FA697B689A42C4D3BA697B689A42C0D3C1
:1031E000FB69181CBD4608B080BDC04680B588B0DC
:1031F00000AFF860B9607A600023FB610023BB6117
:1032000003E0FB68181CFFF775FEFB68181C04211F
:10321000FFF72CFE031C002BF3D1FB68181C0321C5
:10322000FFF75AFEFB68181CFFF748FE031C072B2C
:1032300045D9BB687B6139E0FB68181C0221FFF7A8
:1032400015FE031C012B0CD1BA697B689A4208D287
:10325000FA683F4B101C191CFFF758FEBB6902337C
:10326000BB61FB68181C0121FFF714FE031C012B36
:1032700001D1002368E00DE0FB68181CFFF73AFE5F
:10328000031C1A1C7B691A807B6902337B61FB6912
:103290000233FB61FB68181C0421FFF7E7FD031CE8
:1032A000012B03D1FA697B689A42E5D3BA697B683E
:1032B0009A42C1D3FA697B689A42BDD343E0BB68A6
:1032C0003B6138E0FB68181C0221FFF7CFFD031CAF
:1032D000012B0BD1BA697B689A4207D2FB68181C94
:1032E000FF21FFF713FEBB690133BB61FB68181CAC
:1032F0000121FFF7CFFD031C012B01D1002323E0A7
:103300000DE0FB68181CFFF7F5FD031CDAB23B6902
:103310001A703B6901333B61FB690133FB61FB6858
:10332000181C0421FFF7A2FD031C012B03D1FA692D
:103330007B689A42E5D3BA697B689A42C2D3FA693C
:103340007B689A42BED3FB69181CBD4608B080BD9D
:10335000FFFF000080B582B000AF78600A1CFB1C44
:103360001A70FB1C1B78002B05D07B68181C0021F1
:10337000FFF7F2FD04E07B68181C0421FFF7ECFD69
:10338000BD4602B080BDC04680B586B000AF786053
:1033900039607B68181CFFF73DFE031CBB600023EF
:1033A0007B6101235B423B610223FB6018E07B6988
:1033B0000133FA685343B868191CFEF7EDFF031C8C
:1033C0003B613A693B689A420AD97B6901337B6168
:1033D0007B69FF2B04D900237B61FB680233FB6010
:1033E0003A693B689A42E2D879687A69FB68081CB6
:1033F000111C1A1CFFF734FEBD4606B080BDC04646
:1034000080B582B000AF78607B68181CFFF7B6FD0E
:10341000031C181CFFF7E2FC7B68181C0121FFF756
:10342000E1FD7B68181CFFF7C3FD031C181CFFF7A8
:10343000C1FC7B68181C0021FFF78EFD7B68181CFF
:10344000072100220023FFF76FFD7A68034B101C51
:10345000191CFFF799FFBD4602B080BDA086010090
:1034600080B584B000AF78600B4A8E239B00D258A1
:10347000FF231340FB607A68FF231340FA6813436D
:10348000FB60054AFB68ED21090219438E239B006E
:10349000D150BD4604B080BD0080044080B584B0EA
:1034A00000AF78600C4A8E239B00D258FF23134054
:1034B000FB607A68FF231340DA43FB681340FB602C
:1034C000054AFB68ED21090219438E239B00D15068
:1034D000BD4604B080BDC0460080044090B583B0B6
:1034E00000AF021CFB1D1A70074A07498023C95808
:1034F000FB1D1B780120041C9C40231C19438023C6
:10350000D150BD4603B090BD0080044080B582B06C
:1035100000AF7860034A98237968D150BD4602B065
:1035200080BDC0460080044080B582B000AF7860A6
:103530000A1CFB1C1A70FB1C1A787B681A60BD46BB
:1035400002B080BD80B582B000AF786039607B6822
:103550003A689A60BD4602B080BDC04680B582B070
:1035600000AF786039607B683A68DA60BD4602B0C7
:1035700080BDC04680B582B000AF78607B68DB68F4
:1035800080221A437B68DA60BD4602B080BDC04627
:1035900080B582B000AF78607B68DB688022191C40
:1035A00091430A1C7B68DA60BD4602B080BDC0460C
:1035B00080B582B000AF7860FB1C1970BB1C1A701C
:1035C000FB1C1A787B681A60BB1C1A787B685A60EF
:1035D000BD4602B080BDC04680B582B000AF786005
:1035E0007B685B69181CBD4602B080BD80B582B0A7
:1035F00000AF78600C20FFF771FF0120FFF786FF16
:103600007B68181C0721FFF79DFF7B68181C0321AE
:10361000FFF7A4FF7B6810229A62BD4602B080BD0E
:1036200080B586B000AFF860B9607A6000237B6136
:10363000BB683B610CE03B691B78FA68101C191CE5
:10364000FFF772FF3B6901333B617B6901337B61AB
:103650007A697B689A4207DAFB68181CFFF7BCFF9F
:10366000021C20231340E6D17B69181CBD4606B01E
:1036700080BDC04680B588B000AFF860B9607A60A0
:103680000023FB61BB68BB6115E0F968BA697B6820
:10369000081C111C1A1CFFF7C3FF031C7B617A680E
:1036A0007B69D31A7B60FA697B69D318FB617B69FC
:1036B000BA69D318BB617B68002BE6DCFB69181C78
:1036C000BD4608B080BDC04680B586B000AF78600A
:1036D0003960FFF7B7FA031C7B613B681B0178690F
:1036E000191CFEF759FE031C3B613B691B0AFB607A
:1036F000FB681B023A69D31ABB607B68181CFFF792
:1037000039FFBB68DAB2FB68DBB27968081C111CB0
:103710001A1CFFF74DFF7B68181CFFF739FF78690B
:103720003969FEF739FE031C181CBD4606B080BD82
:1037300008B50020011C021C00F094FDFEF7C8FD36
:1037400008BD08B502F0C5FC08BD08B502F0D7FCFD
:1037500008BD41180B78342B01DC00201CE0352B10
:1037600006D10B1C01331A78302AFBD0002AF4D082
:103770000B1C013B1A78392A02D130221A70F8E763
:1037800001321A700378302BE7D00B1A03D40B7870
:1037900001398B70F9E70120704770B5051C0C1CCE
:1037A0008E1FB4420CD0281C0A21FEF7EDFD0A231F
:1037B0005B4243433035ED18013C6570051CF0E772
:1037C00070BD0000000000000EB410B591B013AB46
:1037D00004CB041C0021282206A80593FFF7B5FF9F
:1037E0000A230993124B059A0893139B01920093A5
:1037F000104B06A802930D4B0B4A069400F084FD73
:10380000089B041C013B0893002B03DB069A002352
:10381000137003E0002006A901F08CFC201C11B0FD
:1038200010BC08BC03B01847FFFFFFFFFFFFFF7F7E
:10383000FFFFFF7F39380000F0B50E684C68A5B077
:1038400007920A93321C231C0C920D930B900D9837
:1038500043005B0D0F930F9D994B9D422AD10203AC
:10386000079C051C0C980023120BE37002436E2387
:10387000002A14D16922637066232270A370002D80
:1038800003DA904B2A9C236011E00A9DAD0704D413
:103890000A9C640708D58C4B07E08C4B05E0079C1D
:1038A000612223706270A370894B2A9D2B600320D4
:1038B00000F080FC0B9D20239D432B1C0025412BF9
:1038C00000D15AE2301C211C704B6F4A02F03AFBC7
:1038D000A84205D08020000601252418109500E09C
:1038E0001090301C211C694B674A02F00FFB002826
:1038F00000D021E217AA211C301C01F02DFD179CDD
:10390000189019912E20FF30604372494018FA2117
:103910008900FEF739FD021B08905D485D4901F002
:103920005BFD089C22902391002C05DA5A4A5B4BE0
:1039300064421E921F9307E0089D594A594B1E92FC
:103940001F93002D16D02C1CE00709D5229823992F
:103950001E9A1F9B01F070FF22902391012C09D029
:103960001E981F991E9A1F9B01F066FF64101E90FF
:103970001F91E9E718981999229A239B02F020F8E1
:103980001A901B911A981B99474A484B02F0DAFA91
:10399000002813D01A981B99454A464B01F04CFF5A
:1039A000434A444B089C1A901B9122982399013C4E
:1039B000089402F005F822902391E3E71A981B99E6
:1039C0003D4A3E4B02F036FB002813D01A981B9953
:1039D000374A384B01F0F4FF354A364B089D1A90B0
:1039E0001B91229823990135089501F025FF22901B
:1039F0002391E3E71A981B9902F02AFA089C099090
:103A000063421194002C00DA1193099802F073FAC2
:103A1000179B089DEA1A01F0DFFC1C4B1A4A1A900A
:103A20001B911C921D93002D56DA1B481B491E90BA
:103A30001F91209221931E9E1F9F1E981F99002662
:103A4000321C3B1C02F06CF8209C219D021C0B1CBC
:103A5000201C291C02F058F9114A124B2090219188
:103A60001E961F971E981F9901F0E6FE021C0B1C64
:103A70000748084902F054F8094A0A4B01F0A0FF30
:103A80002090219132E0C0460000000000000000BC
:103A9000000000000000F03F9A9999999999C93F58
:103AA000000000000000144000000000006AF84020
:103AB00000000000000024400000000080842E412F
:103AC000FF0700001E640000EE630000EC630000CE
:103AD0007764000084EAFFFF089CC449C2481E9036
:103AE0001F9120922193002C00D17FE0119D0E9513
:103AF0000E9CE40743D51A981B99209A219B1C9C85
:103B00001D9D129413951E9C1F9D209E219F01F0C8
:103B100093FE321C149015913B1C201C291C02F0B2
:103B2000F3F8021C0B1C1298139901F085FE021C7D
:103B30000B1C1498159902F0E7F81C901D911A9827
:103B40001B991E9A1F9B01F077FE1A901B911A9EDB
:103B50001B9F1A981B990026321C3B1C01F0E0FFAA
:103B60001C9C1D9D021C0B1C201C291C02F0CCF867
:103B70000E9D1C901D911A961B97012D36D0209EEC
:103B8000219F1E9A1F9B101C191C209C219D02F036
:103B9000BBF8221C2B1C02F0B7F8021C0B1C301CBB
:103BA000391C01F049FE209021911E981F991E9A00
:103BB0001F9B01F041FE1E901F911E9E1F9F1E988D
:103BC0001F990026321C3B1C01F0AAFF209C219D5E
:103BD000021C0B1C201C291C02F096F80E9C209045
:103BE000219164101E961F970E9481E71A981B99D5
:103BF000189A199B02F0E2F9002803D1099D013DB2
:103C0000099502E7189819991A9A1B9B01F088FFE9
:103C100018901991189819991C9A1D9B01F080FF12
:103C20001890199118981999229A239B01F0C8FEAF
:103C30006F4A704B189019911898199901F0FCFD72
:103C4000189019911898199902F002F9189E199F65
:103C5000041C02F050F9021C0B1C301C391C01F032
:103C60005FFF634A634B01F0E7FD189019911898C4
:103C7000199902F0EDF8061C002E03DA5E48013CAB
:103C80003618F9E75D4B9E4203DD5D490134761835
:103C9000F8E7002C05DA099D574A013DA41809955B
:103CA000F7E79C4205DD099D554801352418099523
:103CB000F7E7099D534B9D4219DC201C5249FEF742
:103CC00063FB099B0A277B43051C1B184E49301CCC
:103CD0000993FEF759FB4D4B5D43434364197C4305
:103CE000089DF3183E1C24185E43013D22E0434B1F
:103CF0000998984226DD0A21FEF746FB0A277F42F3
:103D0000031C7B43EB183C4D09906B43E318181CD4
:103D10000A210E93FEF738FB041C381C60430E99F1
:103D200008186843301805300A21FEF72DFB089D5E
:103D3000061C0135089505E0052300265B42089323
:103D4000341C099607983025011C05700631099826
:103D5000FFF723FD0799201C0C31FFF71EFD079983
:103D6000301C1231FFF719FD079C0023E574089DF4
:103D700023750535109CAD002543E80701D5244B7C
:103D80000AE00A9CA40704D40A9C640703D5214BCB
:103D900002E0214B00E0214B2A9C2B982360012359
:103DA0009D43EB179B0F0B995D19AD1004686129BA
:103DB00011D007DC452900D188E0472967D0412987
:103DC00063D108E00B9A662A00D108E1672A5ED029
:103DD000652A5AD17AE00D9B0F9D1803000B002D28
:103DE00020D00F496B1822E00000000000001440B2
:103DF0000000000080842E4140420F003F420F002F
:103E0000C0BDF0FF9F860100A08601006079FEFF23
:103E10001E640000EE630000EC63000077640000A5
:103E200001FCFFFF0C9A0F9B024300D0C64B002CF5
:103E300010D10A9D2D070DD40B9C612C01D1C349D3
:103E400000E0C3490F9A501E824130320798FFF7B5
:103E5000BBFC11E00B9D612D01D1BE4900E0BE49C4
:103E60000F9A0190551EAA410C9D02933032009585
:103E70000798231CFFF7A8FC0D99002901DBB74B1D
:103E800000E0B74B2A9C236094E167200B900A99CD
:103E900080231B0119430A91002C02DC2B9C012377
:103EA00023602B9C12212368112B00DC591C0798DE
:103EB000FFF74FFC2B9C2D1823689D4200DA88E009
:103EC0002B9C013B23600B9C023C0B942B9C236896
:103ED000112B05DD2D9C113B23602B9C11232360AE
:103EE0002B98802600680A99041C360102340E4083
:103EF00004D10798211CFFF72CFC2D18079A2B984A
:103F0000537813700368002B03D1964B0A9919421A
:103F100003D0079A2E23537000E001242D980368E4
:103F2000002B03DD07993E230B550134002E10D0E2
:103F30000A9A12070DD407980319013B1B78302BFE
:103F400001D1013CF7E73E2BFBD02E3B5A425341B7
:103F5000E41A0B9A0799631C0A550234002D04DAFF
:103F60002D226D42261CCA5403E007982B22261CE2
:103F7000C2547D4B9D420CDDFA21281C8900FEF7BE
:103F800003FA0799031C30330B55784B661C5843D2
:103F90002D18632D0CDD281C6421FEF7F5F9079C14
:103FA000031C3033A35564235B42584301362D185C
:103FB000281C0A21FEF7E8F90A225242031C50434A
:103FC000079C30333035A3552818A3195870B01CFE
:103FD000F0E0281D00DA73E7EA439B1823602B9C6E
:103FE000802322681B01002D51DA6E42511C8E4243
:103FF00009DD079D30232B702E236B7020682D9CCC
:10400000206002243BE05219941C122C03DD2D9CED
:10401000113A226013240A9818420CD10798211CE7
:10402000FFF797FB002806D0EE430134002E02D1A3
:10403000079D6B780DE0079D2B19012E0DD1079D73
:104040005A1B002A03DD1A78013B9A70F7E7013406
:1040500030232B702E236B7011E0079D5A1B002A12
:1040600003DD1A78013BDA70F7E730232B702E233B
:104070006B703C23AB702C9D013E02342E602D9D55
:104080002B68002B75DD079D3E232B5527E0AE18CE
:10409000B41C122C41DD0A981324184207D107984A
:1040A000211CFFF756FB002801D001351424621EA5
:1040B000079B954215DA5A7807991A7001335A1AF4
:1040C000AA42F8DD4B192E225A702B9A2D9B1268AA
:1040D000AD18113D1D60002D4BD03E230B55013412
:1040E00047E05978079819700133191A9142F8DBA3
:1040F00003192D1B2C99013B3C2202351A700D60CF
:104100002E222B9D02552A68631C002A30D02D9D3B
:1041100002342A603E22C2542BE00A98184207D18A
:104120000798211CFFF715FB002801D00135F41C6E
:10413000079B5A7807991A7001335A1AAA42F8DD78
:104140004D192E236B7014E001FCFFFFF06300009B
:10415000F8630000006400000F6400007764000052
:104160001E64000008080000E703000018FCFFFFC1
:104170001C1C0A9D2D0512D50A9D201C2D0719D443
:10418000079D2B19013B1878302801D1013CF7E736
:104190003E28FBD02E3843425841201A0AE02B9D7E
:1041A000201C2B68002B05D10A9C082323405A426F
:1041B0005341C01A25B0F0BDF0B58FB00C1C071CE0
:1041C000161C0021282204A81D1CFFF7BEFA0A2392
:1041D00007930E4B621E06930D4B0024019502932C
:1041E0000096231C04A8049700F08EF8069B051C7B
:1041F000013B0693A34202DB049B1C7003E0201CDE
:1042000004A900F097FF281C0FB0F0BDFFFFFF7F4F
:10421000393800000FB473B506AB20CB68460121D6
:104220002A1C0193FFF7C8FF041E14DD461C301C36
:1042300001F038F9009000280DD0311C2A1C019B98
:10424000FFF7BAFF064B0099D86B221CFEF79CFAC9
:10425000009801F089F9201C76BC08BC04B018470E
:10426000FC00001070B5244CA02200215200201C3C
:10427000FFF76BFAC02001F07FF9204D0021C0222A
:104280002860FFF762FA28680023282218215A4381
:104290005943A218411801335162082BF5D1221C51
:1042A0001749002000F0F0FF802280235B01201CD2
:1042B0000021D20000F0CEFE261C124D2836291C0B
:1042C000321C012000F0E0FF80228023301C5B01C3
:1042D00050340021D20000F0BDFE291C221C022017
:1042E00000F0D2FF80228023201C0021D2005B013D
:1042F00000F0B0FE70BDC046FC000010F8000010D9
:104300002064000022640000F0B5D1B00E920F933B
:104310000024569B579D071C079418785C1C0A9430
:10432000002801D100F092FE0026252825D0079C08
:10433000079E0F990134F317994207DC01D000F072
:1043400072FE0E9AB24201D800F06DFEBB68013BCE
:10435000BB60002B05DB3B685A1C3A60187000F00C
:1043600062FE391C00F0E6FE00F05DFE2B2C0BD93E
:104370002D2C0FD101231E430A920A9B0A9A1C7806
:1043800001322B2CF2D10AE0202C0AD0232C0AD1A6
:104390000823F0E7302C06D180239B00EBE70223B3
:1043A000E9E70423E7E72A2C0CD12B682A1D002B10
:1043B00002DA01215B424E400A98151C4478023013
:1043C0000A9008E00023211C3039C8B20A9209285B
:1043D00001D800F02CFEDA43D217134000210C93D1
:1043E0000B912E2C1CD10A9A14782A2C06D12C68F9
:1043F00004350B94547802320A9209E00A9B221C7D
:10440000303A0133D1B20A93092901D800F016FEDF
:104410000B98002802DB10231E4301E000210B91C2
:104420006C2C0ED10A9A14786C2C05D15478602328
:1044300002321E430A9204E00A9B01330A932023AE
:104440001E434C2C01D0712C04D10A9860230478AF
:104450001E431EE0682C0FD10A990C78682C05D1F8
:1044600080235B004C781E4302311AE00A9A8023B5
:1044700001320A921E4315E06A2C06D140231E43E6
:104480000A9B1C7801330A930CE07A2C04D10A9819
:10449000047801300A9005E0742C03D10A990C7855
:1044A00001310A91672C1EDC652C00DBAAE2472C47
:1044B00000D1A7E209DC412C00D19DE2452C00D1BE
:1044C000A0E2002C00D1B2E027E0612C00D193E201
:1044D00003DC582C00D187E11FE0632C19D0642C39
:1044E00000D138E219E0702C00D1D4E108DC6E2C48
:1044F00000D1A2E000DDD8E1692C00D12BE20CE074
:10450000752C00D1FAE1782C00D198E1732C04D1FC
:10451000B4E02C1D11942C6800E011950C98012337
:10452000013833400890109333D120210B91B2050C
:1045300001D530260B96002500260C9A0798023AE2
:10454000521B43190892002A22DB0798C1172890B2
:1045500029910F98289A299B52197341984203DC9C
:1045600011D10E9991420ED9BB68013BBB60002B63
:1045700005DB3B685A1C3A600B9A1A7003E00B98F3
:10458000391C00F0D7FD01220023AD185E41D4E7AD
:104590000793079E07990F9A0136CB179A4203DCBF
:1045A00010D10E9B8B420DD9BB68013BBB60002B29
:1045B00004DB3B685A1C3A601C7003E0201C391C69
:1045C00000F0B8FD109C0796002C01D100F029FDE9
:1045D000002400250899E343CB4221D4F0172A9602
:1045E0002B900F992A9A2B9B12196B41994203DC4D
:1045F00011D10E9890420ED9BB68013BBB60002BD5
:1046000005DB3B685A1C3A6020221A7003E0202028
:10461000391C00F08FFD01220023A4185D41D9E769
:10462000CB43DB170B40F318079300F0FAFC0A9C0E
:104630001195013C0A9400F0F4FC2B1D11932B689A
:10464000700605D5079CE2171C605A6000F0E9FC73
:10465000B00603D5079C1C6000F0E3FCF00503D511
:10466000079C1C7000F0DDFC300603D5079C1C8005
:1046700000F0D7FC079E1E6000F0D3FC2C1D2D68B7
:1046800011941095002D01D1BF4C1094109800F09A
:1046900005FD041CF00603D50B998C4200DD0C1CB3
:1046A0000C9A0123121B334008920C9337D120231C
:1046B0000B93B00501D530260B9600250026089AED
:1046C000013A531B22D40798C1172C902D910F98B3
:1046D0002C9A2D9B52197341984203DC11D10E99EB
:1046E00091420ED9BB68013BBB60002B05DB3B68E8
:1046F0005A1C3A600B9A1A7003E00B98391C00F0B0
:1047000019FD01220023AD185E41D8E7089EF3434E
:10471000DB173340079ED21AF61807960892002539
:104720000026AC4224DD0798C1172E902F910F98D8
:104730002E9A2F9B52197341984203DC13D10E9984
:10474000914210D9BA681098013ABA604319002A08
:1047500005DB3A68511C39601B78137003E0187848
:10476000391C00F0E7FC01220023AD185E41D8E7B8
:10477000E343079EDB171C4036190C9C0796002C60
:1047800001D100F04EFC00240025089EE343F342D3
:1047900022D4079E0F99F01730963190309A319BB2
:1047A00012196B41994203DC11D10E9E96420ED92B
:1047B000BB68013BBB60002B05DB3B685A1C3A60C1
:1047C00020221A7003E02020391C00F0B3FC0122E3
:1047D0000023A4185D41D8E7F343079CDB1733405F
:1047E000E418079400F01DFC402333400AD007353D
:1047F00007239D43281C083029686A68119004919A
:10480000059204E02A1D2D681192049505938023DA
:10481000334006D0684610210B5A002204930592BB
:1048200006E0F00504D569461020425C0593049229
:10483000310701D5554D00E0554D564A29E040233A
:1048400033400AD0073507239D43281C08302968C8
:104850006A6811900491059204E02A1D2D68119256
:10486000049505938023334006D0684610210B5AE7
:1048700000220493059206E0F00504D56946102055
:10488000425C05930492310701D5434D00E0404D51
:10489000424A9446ABE0281D404A2D680021049509
:1048A0001190059194463C4DC7E0402333400AD017
:1048B000072307359D432B1C08332868696811932B
:1048C0000490059104E0291D2D681191049505932C
:1048D0008023334006D06A461020835A0021049377
:1048E000059106E0F20504D5684610210A5C05939F
:1048F0000492320700D477E0294D76E0402333401C
:104900000AD0072307359D43291C08312A686B68A4
:1049100011910492059304E0281D2D6811900495CF
:1049200005938023334005D069461022535A0493DF
:10493000002305E0F00504D569461020425C04928E
:10494000059310223240124B944675D0154A00212F
:1049500016408C4670E072060AD5072307359D4342
:104960002B1C08332868696811931490159105E091
:104970002B68291D1493DB1711911593320613D55B
:1049800014A80023C35E14E0246400002B6400001C
:1049900077640000336400002E640000446400006B
:1049A00031640000FFFDFFFFF10505D514AA0023C7
:1049B000D3561493DB171593159B002B08DA149A22
:1049C000159B00215042994104900591C84D0CE07F
:1049D0001498159904900591B10703D4720703D573
:1049E000C44D02E0C44D00E0C44D00239C46F006D7
:1049F00023D5C3490E4020E010231E4202D10D21D1
:104A00001E430B918023DB003343F20601D40626BC
:104A10000B96072207359543286869682E1C469037
:104A20004791002100220836049105920022119638
:104A300094461E1C151C00E01D1C079B4395D817AF
:104A400032933390329833990E9A0F9B121A8B41FE
:104A5000089209930B9901235B4244934593429139
:104A60000023552048A958540133202BF9D1822323
:104A7000DB001E4201D101234293672C16DC652C1A
:104A800000DBC9E0472C00D1C6E006DC412C00D198
:104A9000C2E0452C00D0CFE0BEE0612C00D1BBE0ED
:104AA000642C11D0582C00D0C6E010E0702C0ED031
:104AB00005DC692C08D000236F2C21D0BCE0752CBC
:104AC00002D0782C03D0B7E0002410942FE000230C
:104AD0000499059C0B93214300D1AFE004980F216A
:104AE00001406246505C48A9585405980499059ABB
:104AF0000407080904431109049405910133E7E709
:104B0000049A05980B93024300D197E0049807217B
:104B10000140303148AA99540599049A059C4807E8
:104B2000D1080843E208049005920133E8E7109C9D
:104B3000049B05980B94034300D17FE0049A0599E8
:104B40009208141C049A8B071C435208209488086E
:104B5000CB07141C21901C434808229423902298D0
:104B60002399209A219B12184B4114091907201CE4
:104B700008431909189019911898199912184B415E
:104B8000140A1906201C0843190A1A901B911A9836
:104B90001B9912184B41140C1904201C0843190CC2
:104BA0001C901D911C981D9912184B4100212693B1
:104BB00027912698279912184B41D4085907201C91
:104BC0000843D9081690179106240025049A059BDE
:104BD00016981799A4185D410A22002301F062FA81
:104BE000241A8D4120092B07011C19432A091E9103
:104BF0001F92169817991E9A1F9B12184B410A2054
:104C000050430499109C3031081A48A9605401346B
:104C10001094049205938AE743AB009342AB01934F
:104C200044AB029345AB0393201C46A948AA331C0E
:104C3000589CA0470B9001E000240B948023DB00DC
:104C4000334024930DD000234293449B002B01DD7D
:104C5000013B4293459B002B0BDD4298013BC3185F
:104C600003E042990B9C0B1B01D4429301E0249C6E
:104C700042940B98429900254418439800F00EFA8C
:104C80000C9A01233340141B25931E4B241A1094B5
:104C90001E4214D10024002507E00998A84216DC22
:104CA00012D001220023A4185D41109B013B1A1B66
:104CB000F3D5109CE543ED1725405B1B10930023B3
:104CC00000241293139434E00899A142E9D9BB68F7
:104CD000013BBB60002B05DB3B685A1C3A6020227D
:104CE0001A70DEE7391C202000F024FAD9E7C0460C
:104CF0001E640000EE630000EC63000077640000B7
:104D0000FFFDFFFF01020000E8173495359034984D
:104D10003599129A139B12184B410999994216DC46
:104D200012D0012200231298139980185941129031
:104D30001391439B129C5A1C43921B782C190C9480
:104D40009C46002BE0D112E0089C9442E9D9BB6854
:104D5000013BBB60002B05DB3B6860465A1C3A6098
:104D60001870DEE76046391C00F0E4F9D9E72598B1
:104D7000002833D12024B10500D530240025002699
:104D8000109A013A531B21D40C9A0998D3173692E2
:104D90003793369A379B52197341984203DC10D1EE
:104DA000089991420DD9BB68013BBB60002B04DB25
:104DB0003B685A1C3A601C7003E0201C391C00F050
:104DC000B9F901220023AD185E41D9E7109C0C9E71
:104DD000E343DB172340D21AF4181092249E002ECE
:104DE00002D10025002698E000260B98864200DBC1
:104DF000E5E048ABF05C3C2804D03E2865D10020BB
:104E0000002145E0002100220C910D92449B0C9959
:104E1000013B65184493002B6DDBE21739923894FF
:104E2000389839990C9A0D9B12184B41099999425F
:104E300003DC11D1089890420ED9BB68013BBB60DE
:104E4000002B05DB3B685A1C3A6030221A7003E0E5
:104E50003020391C00F06EF90C980D9901220023C6
:104E6000801859410C900D91D0E7E2173B923A948B
:104E70003A983B990C9A0D9B12184B41099999420B
:104E800013DC0FD0012200230C980D998018594192
:104E9000459B0C900D910C99013B65184593002B97
:104EA000E3DA28E008989042ECD9BB68013BBB608C
:104EB000002B05DB3B685A1C3A6030221A70E1E790
:104EC000391C302000F036F9DCE7099A651CE3173D
:104ED0009A4203DC0FD1089BA3420CD9BB68013B6B
:104EE000BB60002B04DB3B685A1C3A60187002E080
:104EF000391C00F01FF901362C1C76E7E1173C94B1
:104F00003D9109983C9A3D9B5219734198420FDCA0
:104F10000BD001220023AD185E41429B6219013B78
:104F20000C924293002BE9DA12E008999142F0D9F1
:104F3000BB68013BBB60002B05DB3B685A1C3A6039
:104F400030221A70E5E7391C302000F0F3F8E0E772
:104F5000002400250B9E211C331B002B2ADD0C9EF8
:104F6000F0173E963F90099E3E9A3F9B12196B4167
:104F70009E4203DC19D10898904216D9BB68013BC8
:104F8000BB60002B09DB3B680B985A1C48AE3A60AB
:104F9000C94332188A5C1A7007E00B9E48AAC943BD
:104FA0009319C85C391C00F0C5F801220023A4182D
:104FB0005D41CFE7F443E41734400C9E3419259E3D
:104FC000002E2BD0002500261099EB43CB4221D494
:104FD000E017409441900999409A419B52197341BE
:104FE000994203DC11D1089890420ED9BB68013B6D
:104FF000BB60002B05DB3B685A1C3A6020221A700C
:1050000003E02020391C00F095F801220023AD18A0
:105010005E41D9E7CB43DB170B40E418079E3619F6
:105020000796119D079C07940A9BFFF776F90A24BF
:10503000634314785B180132FFF7C5F90B9C0A2112
:1050400061438A180B921C78FFF7D9F9079851B081
:10505000F0BDC046F0B5C5680124AE071AD0802661
:10506000B600B2420BD08026F600B24204D08026B1
:10507000A640B2420ED102E0416A231C04E0064E73
:105080005F1E0124B74205D82A4301610160C36154
:10509000C2600024201CF0BDFEFFFF0010B5411CC3
:1050A000820706D00130431E1B78002BF8D1401A2E
:1050B00018E003680C4A9C180C4A9C43144201D126
:1050C0000430F6E7DCB2421C002C0AD0FF24240294
:1050D000821C234205D0FF242404C21C234200D09A
:1050E000021D501A10BDC046FFFEFEFE808080806B
:1050F000C26820239A43436A10B5041CE2605B68CF
:1051000082699A420DD000F0F3F8E268074B134031
:1051100010221343626AE3605368A36123699360BA
:105120002360E268024B1340E36010BDEFCFFFFF46
:10513000BFBFFFFFF8B5514ACB68061C1A400C1CD4
:10514000CA60980602D5081CFFF7D2FFA268E36880
:10515000511C0EDA98050CD4022149428A1AA26029
:10516000902252021343E36023685A1C22601E708F
:1051700081E0434A1D1C1A40022A05D00022A26089
:1051800080221343E36054E03E490B408021090232
:105190008B420AD10021201C00F050FAE1688906F8
:1051A00002D5201CFFF7A4FFE56890235B02F022E4
:1051B0002B431201E36015421ED1606900F0BBFF72
:1051C00000280BD06A0509D5636A23612360012397
:1051D000E36192235B022B43E3600DE080277F01B4
:1051E000381C00F0C9F99423E2685B022B431A4390
:1051F00020612060E761E260902109012268256951
:105200000B4219D0636A99688A4200D9111C491B64
:1052100009D1636A6A1C9A602260E269511EA1602A
:10522000DA602E7027E0281C221C00F005F9002807
:10523000EFD0012040421FE0511CF0B221601070FD
:10524000626A2768916884468F4200D9391CE769F1
:10525000491BD760580504D463460A2B01D0B942D4
:1052600009DB00239560281C2560A360221C00F048
:10527000E3F80028DDD1F0B2F8BDC046FFFFF7FF2C
:105280008A10000010A0000070B50D1C061C101C38
:10529000141C00F081F92B78722B06D0772B07D0E5
:1052A000612B20D10823114A04E00023012201E0F0
:1052B00004230222013529782B2905D0622908D13F
:1052C00004210A43012102E003210A4302210B4386
:1052D000F0E7E26066611A0706D5201C0021022271
:1052E00000F0ACF900E00024201C70BD028000003A
:1052F00038B5436A041C056902689968C368134895
:105300001840E06082201840022802D0012040426C
:105310001AE080204002184016D0914200D2111CA1
:10532000A94209D1636AE2689D60094B00201340DD
:105330002560A060E36007E0491B281C221C00F0E8
:105340007BF80028EED0E1E738BDC046FFFFF7FF4D
:10535000FFFFFEFF00000000F8B5141C194B184AAF
:10536000061C0F1C00F0D2FD002804D0002323608F
:105370001449134823E07A00134D520D301C391C98
:105380005319002A15D13D032D0B321C6F00D60F87
:105390003E43802736033F03360B52003D4205D083
:1053A0000D0D2D05291C3143101C02E0013B351C5D
:1053B000ECE72360054A064B0B40111C1943F8BD6E
:1053C000000000000000000002FCFFFF0000E03FC2
:1053D000FFFF0F80C046C046D0B5141C114B104AC9
:1053E000061C0F1C00F092FD002802D00D490C484D
:1053F00015E07B005B0D1C190B4B301C9C4206DD3D
:105400000A4B22221A600A4B1868596807E0002CE0
:10541000ECDD084B64053B406408191C2143D0BDFA
:105420000000000000000000FE07000068000010FF
:1054300058640000FFFF0F80F7B5D56801900E1C7F
:10544000141C5769EA0205D51023381C1D4300F0CF
:105450006FFEA061114B1D4208D0381CA16900F0FD
:1054600070FE002813DB0E4B1D40E560321C381C1B
:105470000199FDF789F9801B431E98414042430082
:105480005B08F61AA3699E19A661002805D0E26898
:10549000802313430120E3604042FEBD1000020060
:1054A000EFFFFDFFF8B52F4FC51C3C68AD08002885
:1054B0000FD0002606E0216880235B05994215D0B5
:1054C000261CA468002CF6D10C3000F063F9421CB5
:1054D0003CD1002045E01668802149058E4209D163
:1054E000516892685B1803336360A260A2686368C6
:1054F000002AF0D1AB4206DBE91C994203DB802392
:105500009B05236020E0291C0A318B4210D98021A1
:105510008905201C21600C30A90041186560A1603C
:105520005B1B80246405033B0C604B608A6018E0C1
:10553000002AC5D19B00C01A00F02CF90130C8D058
:1055400080239B0523606560201C09E080239B0568
:10555000036045608460002E01D1386000E0B060D7
:105560000C30F8BD3C020010002803D080230C381A
:105570005B0503607047000010B5FFF793FF041E42
:1055800005D104491722FDF7FFF800F0CDFD201CDE
:1055900010BDC04660640000F0B5436AC5688BB0BA
:1055A000041C476906690193AB0726D02B0716D464
:1055B00000F02AF8381C00F0B8FD2B0502D5301C8D
:1055C000FFF7D2FF0F4BAD0DAD059D4207D102A8ED
:1055D000216A202200F0B8FD02A800F0D1F80021D5
:1055E0001822606AFEF7B1F8201C00212822FEF77D
:1055F000ACF8019B0020636201E0012040420BB047
:10560000F0BDC046000080AD38B5002803D000F0E2
:10561000E1F8051C0EE0041C051C0748201800F0EA
:10562000D9F8002801D001256D42A02328345B0061
:105630009C42F2D1281C38BDFC000010F7B53B4B52
:105640000D1CC168041C161C47690091194269D0E1
:10565000381C00F070FD0190002863D1012E04D0A9
:10566000022E07D0002E5DD123E0201C00F062F84E
:105670002D181EE0381C00F05BFDE168002804DAFC
:1056800080231943E16001264DE0626A2668936831
:105690009E4200D9331CA6699B1926699B1B8E0666
:1056A00003D55268934200DA131C834200DA031CCC
:1056B000ED18002D36DB009E636AB60404D522681F
:1056C0009968914200D29A60A1698D420DDB2068F1
:1056D0009A68824200D2021C20695618361AB542D6
:1056E00003DCDF68CE19B54207DB009E00212022D3
:1056F000A160616032435D6010E0009E6D1AB607E4
:1057000001D5EF1BA760009EF60702D5821AAA18E2
:105710006260009A4519202325609A43044B1A4081
:10572000E26001E0022601960198FEBD0300100030
:10573000BFCFF7FFC368990705D1104B2122012085
:105740001A60404218E0202219030BD5134202D000
:10575000436A586804E0036881695A180369D01ADB
:10576000013809E0134202D0436A586804E0036834
:1057700081695A180369D01A7047C0466800001042
:1057800010B5041CFFF78AFC011C201C00F0D6FC9D
:1057900010BD000070B50C4C2368002B01D10B4BE1
:1057A0002360C61C256803239E43AE19301C00F0FD
:1057B00035F8002802D12660281C04E0044B0C2296
:1057C00001201A60404270BD4002001044020010E7
:1057D00068000010C36870B5041C032018401AD07C
:1057E0009A0605D5636A201C5D68FFF781FC04E01A
:1057F0002368A2699D182369ED1AE268064B201CF4
:105800001340E360FFF774FD291C061C0022201CD6
:10581000FFF714FF301C70BDFFCFFFFF044B002BC0
:1058200004D0002298425241101C00E0181C70471E
:105830000000000000000000F0B58BB01F1C0092BB
:1058400001934B000D1C049005915B0D00D181E08C
:1058500053498B4200D17DE07A00520D7AD08A42C2
:1058600078D0D2183B1C6B40DB0FDB07009803930A
:1058700080242B031B0B64031C430892FE02420D81
:10588000802316431B061E430021221C301C0B1CC8
:1058900000F008FC069007910099201CCD02002121
:1058A0002A1C0B1C00F0FEFB09910021041C049A29
:1058B000301C0B1C00F0F6FB009001910021281C0D
:1058C000049A0B1C00F0EEFB009A019B8446081C16
:1058D0000021261C0F1C36184F41B6185F41099A4B
:1058E0003C1C0D1C0B1C12196B4164460698079951
:1058F00012184B41A1082B48089C0E4321182A4836
:1059000098420AD329481D1C2118141CA4185D4173
:10591000F00F221C02432B1C7600F40F00251219F5
:105920006B418020141C0006864201D10120844373
:105930001F48814205D80A050399201C0B43D11842
:1059400027E0002903DB1B4B039C234300E0039B60
:10595000191C1DE03A1C6A401749D20FD2076B0090
:105960008B4204D87800884204D8111C10E01349F7
:105970008B4207D111487900814203D85B0D01D0D9
:10598000490D02D10549044803E00A4B191C114393
:1059900000200BB0F0BDC046000000000000F87F02
:1059A000FF07000001FCFFFFFFFF0F0000FCFFFFEF
:1059B000FD0700000000F07FFFFFDFFF0000E0FFB9
:1059C000F0B50D1C87B06E00049005910292039310
:1059D000191C760D5FD04C4A96425CD05B005B0D83
:1059E00059D0934257D00A1C6A40E802049D029F96
:1059F000CC02F61A80216B0D184309067B0D1C435F
:105A00000B1C00920343EA020C43FD029C4202D8A5
:105A100003D1954201D93D4906E0DF0759085008F6
:105A20000B1C3A1C3A490243E707680876183843CA
:105A30006108352500246400994206D801D19042BE
:105A400003D80127121A8B413C4392185B416F1E09
:105A5000212D02D101943D1CEDE73D1EEBD1994271
:105A600008D801D1904205D8019D013463426341B9
:105A7000ED1801950099274BCF0FFF079E4204D8E0
:105A80003605019DF71979191EE0002E01DB224E23
:105A90003743391C2AE0214F6E00BE4228D84A0005
:105AA000BA4225D80B1C2B435B005B0D5B0503D171
:105AB00012491148181C1DE00B1C6B40DB0F740DC4
:105AC000DB07640502D1191C201C13E0540D64058A
:105AD00003D1114A111C1943F6E7BA4203D00E4A0A
:105AE000111C194302E0964202D0191C002001E06B
:105AF0000348044907B0F0BD000000000000F87F33
:105B0000000000000000F87FFF070000FD03000018
:105B1000FE030000FD0700000000F07F0000E0FF32
:105B2000F0B587B002900391039F1D1C0092019372
:105B3000049005913A1C9C46049E009B6A4006D541
:105B400080263606AB19009A00F0DEF8C9E0AF42B5
:105B500003D39E420AD8AF4208D180200006039F9B
:105B600012185740049B6A40009E944661460A0DF5
:105B7000614862493C0DA21A2140814200D1A3E054
:105B80008A4200D19AE0604601033F03802040032F
:105B90003F0B090B074301431F2A50D8081CD04074
:105BA0003F1A2025181CD040AA1A91400843301AE9
:105BB0008642B6417642191CBF1B9140061C002943
:105BC00005D0013E731C5A4253414942FF1AC0237B
:105BD0005B031F4251D1F30FC90F76007F000E43C4
:105BE0001F43331C3B4301D0A31E01E0191C52E0AC
:105BF0007A0B05D1320E3F0217433602083BF7E716
:105C00007A0C04D1320F3F0117433601043BFA0CE2
:105C100004D1B20FBF001743B600023B3A0D04D1C6
:105C2000F20F7F0017437600013BE40ADA0A944240
:105C300002D11B05D91953E0E107002051E0352AB4
:105C40001BD8151C203D081CE840301A8642B6417E
:105C50007642BF1B4026B21A91401A1CEA401143FB
:105C60001B0602D0FF23194302E0061C002904D0C2
:105C7000461E434243414942FF1AFB020DD4013CF8
:105C8000630507D0F30F7F001F437600CB0F1E4341
:105C9000490002E02105181C23E0194B24051F4090
:105CA000002909DA013673427341FF1880231B066D
:105CB000994201D101239E43391911E0114B9A42B7
:105CC00002D8111E09D00AE03B0302D0074906485A
:105CD00007E0002A03D106480649101C01E0391CE0
:105CE000301C07B0F0BDC046000000000000F87F87
:105CF000000000000000F87FFF070000FFF7FFFF33
:105D0000FFFFEFFFFE070000F0B587B002900391A0
:105D1000039F1D1C00920193049005913A1C9C4620
:105D2000049E009B6A4006D580263606AB19009A71
:105D3000FFF7F6FE7DE0AF4205D2039F049B57407C
:105D4000009E6A4094463E493E4A380D01409142C9
:105D500068D06446220D821A8A425AD021033F033A
:105D6000802464033F0B090B274321431F2A10D8CB
:105D70000C1CD4403F1920251C1CD440AA1A914069
:105D8000214376188E42894149427F18191C91405F
:105D900014E0352A12D8141C203C0D1CE54076195D
:105DA000AE42AD416D427F194025AA1A91401A1C9E
:105DB000E24011431B0601D0FF231943BB0218D553
:105DC000013673427341FF18002901D102239E431B
:105DD00002057B089B181C4A5900914205D8760899
:105DE000FF07301C191C384323E0431C1905002011
:105DF0001FE00138002909DA013673427341FF18A8
:105E000080231B06994201D101239E430305F91803
:105E10000EE00E4B9A4205D8002A08D1FF0FF90771
:105E2000101C06E03B0302D00449034801E0391C82
:105E3000301C07B0F0BDC046000000000000F87F35
:105E4000FFF7FFFFFF070000FFFFDFFFFE07000077
:105E50000B1C400DC90208438021090610B50B4CEC
:105E60000843190D611AC840FF290ED9E024E40047
:105E70004042214209D00020590006D504495C0067
:105E80008C4202D8D80F034BC01810BD1E0400006E
:105E90000000E0FFFFFFFF7F10B5002802D1031CC8
:105EA000021C25E0030C01D1000402E080235B0406
:105EB000C918030E01D1000202E080231B04C91897
:105EC000030F01D1000102E08023DB03C918830F17
:105ED00001D1800002E080239B03C918002801DB68
:105EE000400002E080235B03C918C4126318420516
:105EF000101C191C10BDC10F08B5C90700D04042C5
:105F00008023DB05C918FFF7C7FF08BDF7B50D1CD7
:105F1000009201931F1C9C466B000C1C009A011CF4
:105F2000184304D17D0015430120002D07D0002027
:105F3000644504D1914202D1014A9A424041FEBDDA
:105F40000000E0FFF0B585B00D1C009201931A1C13
:105F50008C46029003911F1C191C2A43164B0ED429
:105F60007A0000209A4224D80120AF4221D8002094
:105F7000AF421ED1029A009B9A42804118E06A000B
:105F800000209A4215D87C009C4212D8029B1A43EA
:105F9000824203D1009A144384420AD001208C45E6
:105FA00007D800208C4504D1009B029A934280417F
:105FB000404205B0F0BDC0460000E0FFF0B587B03C
:105FC000009201930D1C049005910E1C01990498F8
:105FD000029203930A1C8446029F2A43144B0CD45A
:105FE0004A0000249A421FD80124A9421CD8002448
:105FF000A94219D18742644116E06D0000249D42F8
:1060000012D8019842009A420ED801248E420BD831
:1060100001D1BC4508D2049900240D43A54203D107
:10602000029B1A4354425441201C07B0F0BDC046A5
:106030000000E0FFF0B585B0029003910D1C0C1C30
:10604000029900920193181C1F1C28436B008C4678
:10605000009A134D00280CDB0020AB421ED8012013
:10606000BC421BD80020BC4218D163469342404139
:1060700014E00020AB4211D87E00AE420ED80120C1
:10608000A7420BD801D1624508D2029900200B43E8
:10609000834203D1009B33435842584105B0F0BDC1
:1060A0000000E0FF10B543435143C918040C130C22
:1060B0005C43091992B2040C544380B243435043E9
:1060C0002204240C801861411A041B0C80185941C9
:1060D00010BD8446830708D18B0706D1131F04D354
:1060E00004C904C0043BFBD21A1D524205D0891AD0
:1060F000801A8B5C83540132FBD160467047844622
:10610000043A09D3830707D109060B0A19430B0C7C
:106110001943043A02C0FCD2043203D001700130AA
:10612000013AFBD160467047FEE7012040427047CC
:106130000120404270470120404270470120404208
:1061400070470120404270470120404270470000E4
:106150000D0A536F636B65743A256420506F727437
:106160003A25640D0A0000002A0D0000300D0000E1
:10617000720D0000660D0000800D00008C0D000007
:106180009A0D0000C40D0000EA0D0000240E00006E
:106190002A0E0000340E0000A00E00003E0E00008B
:1061A0004C0E0000740E0000D80E0000E20E00003D
:1061B000EC0E0000FA0E0000080F0000120F0000A5
:1061C00025643A536F636B6574204572726F720D6C
:1061D0000A000000C0A800020D0A3D3D3D3D3D3DC6
:1061E0003D3D3D3D3D3D3D3D3D3D3D3D3D3D3D3DDF
:1061F0003D3D3D3D3D3D3D3D3D3D3D3D3D3D3D3DCF
:106200003D0D0A002057495A6E65742025732045BC
:1062100056422044656D6F73207625642E252E32FC
:10622000640D0A003D3D3D3D3D3D3D3D3D3D3D3D17
:106230003D3D3D3D3D3D3D3D3D3D3D3D3D3D3D3D8E
:106240003D3D3D3D3D3D3D3D3D3D3D0D0A00000098
:106250003E3E205735353030206261736564204CF6
:106260006F6F706261636B204578616D706C650D56
:106270000A0000000D0A3D3D3D3D3D202573204EA6
:10628000455420434F4E46203A2044484350203D39
:106290003D3D3D3D0D0A00000D0A3D3D3D3D3D208B
:1062A0002573204E455420434F4E46203A205374C8
:1062B00061746963203D3D3D3D3D0D0A00000000D5
:1062C0000D0A4D41433A20253032583A2530325894
:1062D0003A253032583A253032583A253032583A39
:1062E000253032580D0A000049503A2025642E25E9
:1062F000642E25642E25640D0A00000047573A20BD
:1063000025642E25642E25642E25640D0A000000C8
:10631000534E3A2025642E25642E25642E25640DC7
:106320000A000000444E533A2025642E25642E2591
:10633000642E25640D0A000057495A4348495020ED
:10634000496E697469616C697A6564206661696C1B
:106350002E0D0A00020202020202020202020202E0
:1063600002020202001BB70000010100151718000D
:10637000000101000002010000030100000401000F
:106380000005010000060100000B010100120100E0
:1063900000130100000401000005010001161000B7
:1063A000011410000117100001151000000000007A
:1063B000C027090090051000C05C1500F0B31A005A
:1063C000200B2000009F2400E0322900C0C62D00D1
:1063D00050973100E06735007038390000093D0002
:1063E0004016400080234300C03046002B002000B0
:1063F000307825637025640030582563502564008B
:10640000307825632E252E2A6C6C78702564003038
:106410005825632E252E2A6C6C58502564002D00BB
:1064200072007700286E756C6C2900305800307847
:106430000030003031323334353637383941424359
:1064400044454600303132333435363738396162AD
:106450006364656600000000FFFFFFFFFFFFEF7F42
:106460002A2A2A205F437379735F616C6C6F632003
:086470006661696C65640A00B5
:106478000102573535303000690B0000710B000000
:10648800790B0000810B0000890B0000A10B0000B4
:10649800000000000000000000C000000008DCABA5
:1064A800CDFFC0A80051FFFFFF00C0A800010808E9
:0464B80008080100CF
:040000030000017187
:00000001FF
